:020000022000DC
:1060000000000120D1620200F9620200FB6202007E
:10601000FD620200FF620200016302000000000056
:106020000000000000000000000000000363020008
:10603000056302000000000007630200096302001C
:10604000198F02000B630200E99502000B63020046
:106050000B6302000B6302002D9302000B6302002E
:106060000B6302000B6302000B6302000B63020070
:106070000B6302000B6302000B6302000B63020060
:106080000B630200417B02000B6302000B63020002
:106090000B6302000B630200C1B802000B63020035
:1060A0000B6302000B6302000B6302000B63020030
:1060B0000B6302000B630200000000000000000000
:1060C0000B6302000B6302000B6302000B63020010
:1060D0000B6302000B6302000B6302000000000070
:1060E00000000000000000000000000000000000B0
:1060F00000000000000000000000000000000000A0
:10610000000000000000000000000000000000008F
:10611000000000000000000000000000000000007F
:10612000000000000000000000000000000000006F
:10613000000000000000000000000000000000005F
:10614000000000000000000000000000000000004F
:10615000000000000000000000000000000000003F
:10616000000000000000000000000000000000002F
:10617000000000000000000000000000000000001F
:10618000000000000000000000000000000000000F
:1061900000000000000000000000000000000000FF
:1061A00000000000000000000000000000000000EF
:1061B00000000000000000000000000000000000DF
:1061C00000000000000000000000000000000000CF
:1061D00000000000000000000000000000000000BF
:1061E00000000000000000000000000000000000AF
:1061F000000000000000000000000000000000009F
:1062000010B5054C237833B9044B13B10448AFF3F0
:1062100000800123237010BDA8230020000000008F
:1062200094C90200084B10B51BB108480849AFF3E8
:1062300000800848036803B910BD074B002BFBD052
:10624000BDE81040184700BF0000000094C90200DC
:10625000AC230020A023002000000000154B002BE1
:1062600008BF134B9D46A3F5803A00218B460F468D
:106270001348144A121A05F0E0FC0F4B002B00D013
:1062800098470E4B002B00D09847002000210400B7
:106290000D000D48002802D00C48AFF3008005F037
:1062A0009BFC2000290004F023F805F081FC00BFCE
:1062B00000000800000001200000000000000000B5
:1062C000A8230020B82C00200000000000000000DF
:1062D0000649074A074B9B1A03DD043BC858D050B8
:1062E000FBDC02F0D3FAFFF7B9FF00008CCA020012
:1062F000F0220020A8230020FEE7FEE7FEE7FEE7ED
:10630000FEE7FEE7FEE7FEE7FEE7FEE7F0B595B045
:10631000002415460F4608461E4602F05DF9384631
:10632000234605A9082208951A9D0D9509960A94F9
:106330008DF82C400C9402F0A9F99DF81430079DBB
:10634000BDF81800BDF81A108DF8114003F00302D3
:10635000012A0295ADF80C00ADF80E1028D0022AE3
:1063600004D0384602F03CF915B0F0BDBDF8165027
:10637000C3F3C2038DF81030C5F389150826082D24
:106380002C4628BF08243346224638460EA902F080
:106390007DF92D1B21460EA802AA08AB264400F069
:1063A00005FD002DEBD1384602F01AF915B0F0BD0D
:1063B000BDF81460059DC6F38316C3F3C204B20092
:1063C0000EA9384608238DF81040C5F3952502F034
:1063D0005DF908AB0093284632460EA902AB00F0E7
:1063E0003FFCBEE7014B01221A707047C423002016
:1063F000704700BF00B583B0044B0093044A4023AC
:10640000FFF784FF03B05DF804FB00BF15640200D2
:10641000C823002038B50E480E4D03780E4CEB5CB7
:10642000002525706BB90C30D2B203F037FB08B1F0
:1064300000F08EFF094B1B7813B12378002BFCD0A2
:1064400038BD0430D2B203F0DFFD0028F0D1F1E70F
:10645000F0220020B42C0020C4230020C5230020FB
:1064600030B51648164A0378D35C89B00BBB0C30A4
:1064700003F0A8FA134D0FCD6C460FC495E80F003A
:10648000062584E80F004FF0FF334FF0EB740B4804
:10649000009569460022019302930393069402F04B
:1064A000BFFC08B100F054FF074B00221A7009B07E
:1064B00030BD043003F00AFDDCE700BFF02200200D
:1064C000B42C002078BC0200C523002030B5104D4C
:1064D0000FCD89B06C460FC495E80F00062584E8FF
:1064E0000F004FF0FF334FF0EB740A480A4A009553
:1064F0006946019302930393069402F091FC08B15C
:1065000000F026FF054B01221A7009B030BD00BF14
:1065100078BC0200F0220020E5630200C5230020C1
:1065200008B5FFF7D3FF0448042100F053FB034BE9
:1065300001225A7108BD00BF74CA02000423002062
:1065400070B52F4C84B004F5836001F0FFFB04F2BA
:10655000144001F0FBFBA268D5B2AB1C04EB830135
:10656000081D097911F0040116D0037803F0030324
:10657000012B36D0022B0CD14388C3F3891302338D
:106580001A44D5B2AB1C04EB8303181D197901F032
:1065900004010029E9D1AB1C04EB8303511C5868AA
:1065A0000190C9B204EB810300F00300DB680293A1
:1065B000012802F102041AD0022816D1BDF80630D3
:1065C000BDF80A50C3F38913033304EB93040C4E54
:1065D00006F2144001F0C8FB00B1B460284604B0D4
:1065E00070BD0388C3F38313C9E70025EFE7BDF847
:1065F0000430BDF80A50C3F383131C44E7E700BF1F
:1066000008240020064B074810B500221A7001F03C
:106610009BFF044610B9044802F0ACF8204610BDB8
:1066200008240020E8C90200D0BC020021B9114BA7
:1066300003EBC0000068704730B40F4A0D4C121BCA
:10664000D2080CD00D4D2B88834210D0002303E0DC
:1066500035F82310814205D001339342F8D1002050
:1066600030BC704704EBC300006830BC7047204664
:10667000FAE700BFFCC9020074CA0200A42300208C
:10668000094B013903EBC00003290BD8DFE801F007
:10669000020806040220704740797047007970476D
:1066A0000420704700207047FCC902002DE9F04724
:1066B000944DAA686B689A4284B000F0D1800023A0
:1066C000C5F81834BFF34F8FAA68D3B2023305EB75
:1066D00083010C1D097948071ED56E682F46237863
:1066E00003F00303012B48D0022B04D16388C3F3CA
:1066F000891302331A44D3B20233D5F81804DFF8F1
:1067000004E207EB83010C1D002840F0AD809642A7
:1067100039D909794907E2D405EB8303511C58683C
:106720000190C9B205EB810300F00300DB6802931E
:10673000022802F10204734F2AD0012800F097804A
:10674000D5F810443CB1236820469B689847E3681D
:106750001C68002CF7D16C4B6C486D49181AC008A6
:10676000000440F0020000F0D7F8AB686868181A1F
:1067700018BF012004B0BDE8F0872388C3F383135A
:1067800002331A44B7E7CEF8086004B0BDE8F087DA
:10679000BDF806305F48C3F38918B8F1500FC24600
:1067A000A8BF4FF0500A6AF38F130AF10801ADF841
:1067B000063001F0CBFE06460028C1D06FEA04097E
:1067C0005FFA89F909F1010901F006FF4FEA890929
:1067D00001A930460822002301F022FFCA45E1B298
:1067E00040F28480C9EB0A0A07EB81010C31304684
:1067F0004A4608235FFA8AFA01F012FF30465246F1
:1068000007F10C0109F1080301F00AFF08F1030781
:1068100004EB9707D5F81834D5F81044002B61D154
:106820005CB1E3685A79204631461AB123681B6887
:106830009847E3681C68002CF3D1304601F0D0FE85
:1068400004A8002300F80D3D00F0E4FFD5F818344B
:106850002C4A03B997609DF8030001F003F884E720
:10686000002004B0BDE8F087D3B2023354E7BDF88E
:1068700004302848C3F38312062A28BF0622911C3D
:1068800062F389138900ADF8043001F05FFE06461B
:1068900000283FF455AF01F09FFE0023304601A9C8
:1068A000082201F0BDFEBDF8043013F4707F26D03D
:1068B0004FF000094FF00808E1B205EB81014346B3
:1068C0000C313046042201F0ABFEBDF8043009F172
:1068D0000109C3F38313671C4B4508F104083C46C8
:1068E000EAD897E7304601F07BFE3EE707EB8101EF
:1068F00052460C313046082301F092FE86E72746C7
:1069000088E700BF0824002024CA0200FCC9020056
:10691000B8BC0200E8C902002DE9F04182B002AB28
:10692000002203F8012D2F4C064618460F4600F0B2
:1069300071FFA368656803F580735B1B012B4FD85B
:106940000121294801F0E6F9FFF7FAFD0146264842
:1069500001F0E0F9A368626803F580739B1A012BCC
:10696000EED94FF00108D2B204EB820248F00403E2
:106970006FF38913D36063689DF807000233636087
:1069800000F070FF1848002101F09CF980F310001E
:1069900005EB0803DBB2EDB2320C04EB83030235E6
:1069A00004EB850542EA0040D8602B7966F3C50305
:1069B0002B71AB886FF38913AB806A6867F39F22F2
:1069C000134668F301036FF382036A602B71237827
:1069D0001BB1FFF76BFE0028FBD102B0BDE8F081D0
:1069E0002A46BEE708240020242800202DE9F04391
:1069F00083B002AB002403F8014D334C0646184621
:106A00000F46904600F006FFA368656803F58073A3
:106A10005B1B022B55D801212C4801F07BF9FFF7B5
:106A20008FFD0146294801F075F9A368626803F5F6
:106A300080739B1A022BEED94FF00109D2B204EBFE
:106A4000820249F0040369F38913D36063689DF8F7
:106A500007000333636000F005FFAB1CDBB204EBFF
:106A600083031A48C3F80C80002101F02BF980F34E
:106A7000100005EB0903DBB2EDB2320C04EB83032B
:106A8000023504EB850542EA0040D8602B7966F3B5
:106A9000C5032B71AB8869F38913AB806A6867F310
:106AA0009F22134669F301036FF382036A602B711F
:106AB00023781BB1FFF7FAFD0028FBD103B0BDE836
:106AC000F0832A46B8E700BF0824002024280020CD
:106AD0002DE9F04F83B002AC002504F8015DDFF82A
:106AE000F090054620461F460E46904600F092FE66
:106AF000D9F80830D9F8044003F580731B1B032B29
:106B000062D80121314801F005F9FFF719FD01466E
:106B10002E4801F0FFF8D9F80830D9F8042003F521
:106B200080739B1A032BECD94FF0010AD2B24FF0BD
:106B3000020B09EB82024AF004036BF38913D36062
:106B4000D9F804309DF807000433C9F8043000F088
:106B500089FE04EB0B02E31CD2B2DBB209EB82022A
:106B600009EB83031948C2F80C800021DF6001F0B3
:106B7000A9F880F3100004EB0A03DBB2E4B22A0C9C
:106B800009EB83035C4409EB840442EA0040D860CB
:106B9000237965F3C5032371A3886BF38913A3805D
:106BA000626866F39F2213466AF301036FF3820360
:106BB0006260237199F800301BB1FFF777FD002860
:106BC000FBD103B0BDE8F08F2246ADE724280020BA
:106BD0000824002030B4174DD5F8104400215CB1D2
:106BE000E3681A798A4204D117E0DB681A798A428D
:106BF00013D01B68002BF8D1C3680E4A1971D5F861
:106C0000103493B1DC68C36824681C60D2F8103477
:106C1000DB681860084630BC704701310A29DED1B4
:106C20004FF0FF31084630BC7047C2F81004C2680C
:106C30001360EFE70824002038B5084BD3F8104460
:106C400001251D704CB1E3685D71236820465B68C7
:106C50009847E3681C68002CF5D138BD0824002053
:106C60002DE9F04784B01D460C9C002394F80C805D
:106C70002373EB8881460E461746002B3BD1297AB9
:106C800005290FD06B7A002B3DD1404BA88853F8D3
:106C900021A00021FFF7CAFC524603463C4920468A
:106CA00001F0DCF8062F0FD8DFE807F0484D535A03
:106CB00004633900B168F06896E80C000091019017
:106CC0004946204601F0CAF82B7A052B05D06B7A8D
:106CD0005BB920462F4901F0C1F8204601F0B2F817
:106CE00084F80C8004B0BDE8F08720462A492B4A7E
:106CF00001F0B4F8EDE7294A009220462849294AD4
:106D000001F0ACF8BBE7A888FFF7BAFC264B224994
:106D100053F82020204601F0A1F8297AB5E796E83B
:106D20000C00B168F06837697669039600910190AC
:106D300049460297204601F091F8C5E749462046AA
:106D400001F08CF8C0E749463268204601F086F829
:106D5000BAE74946204696E80C0001F07FF8B3E711
:106D6000B16896E80C0020460091494601F076F89B
:106D7000AAE7B1683069F76896E80C0000910290C4
:106D800049460197204601F069F89DE7DCBC020006
:106D900040BD02004CBD02003CBD020034BD0200FB
:106DA00014BD02002CBD0200F0BC0200082900D96D
:106DB00070472DE9F0471D46002395F80C902B7382
:106DC000D38882B0904607460E46002B67D198F8CC
:106DD0000810052911D098F80930002B67D13B4BDA
:106DE000B8F8040053F821400021FFF71FFC2246A9
:106DF00003463749284601F031F8002405E03A5DA2
:106E0000013401F02BF8082C0AD0A642284631495B
:106E1000F5D828463049013401F020F8082CF4D187
:106E200028462E49DFF8D8A001F018F800240FE01A
:106E3000DAF800201A44527812F0970F14BF1A465D
:106E40002E2227492846013401F008F8082C0DD0DD
:106E5000A64204D93B5D7E2BEAD92E22F1E72846D3
:106E60002049013400F0FAFF082CF1D198F80830DD
:106E7000052B02D098F809305BB928461A4900F072
:106E8000EDFF284600F0DEFF85F80C9002B0BDE86B
:106E9000F08728461549164A00F0E0FFEDE7144A4E
:106EA000009228461349144A00F0D8FF8FE7B8F83B
:106EB0000400FFF7E5FB114B0C4953F8202028464E
:106EC00000F0CCFF98F8081089E700BFDCBC020096
:106ED00040BD020050BD020058BD02005CBD020072
:106EE00060BD020048BD02004CBD02003CBD020076
:106EF00034BD020014BD02002CBD0200F0BC020033
:106F00003423002070B51A4B1D78C0B295B1194BCF
:106F10001C682378984210D004F10802002306E090
:106F200014F833108842164602F1080206D00133E5
:106F3000AB42F5D100231B78FFDE264602F0ECF9C8
:106F40007378A3F10103B3FA83F35B09834200D0A2
:106F500070BD094BD3E900231343F9D1074B08480F
:106F6000196800224908BDE8704000F0E1BB00BF8D
:106F70009829002094290020D02900209029002061
:106F8000B02900202DE9F04F9D4F3B7889B0002BB0
:106F900000F030810025DFF87892DFF87882994E92
:106FA000AA46D8F8004014F8350002F0B5F904EB11
:106FB000C50B14F835409BF80120630814F0010E4E
:106FC000F15CA2F10102B2FA82F24FEA5212A2EB94
:106FD000000014BF0A0901F00F02B0FA80F0400966
:106FE000042A00F2AE80DFE802F074643524030066
:106FF000002800F0AB80BEF1000F14BF0F22F0227A
:1070000001EA020114BF302203221143F1543A78FD
:1070100001359542C5DBD9E90023134306D07A4BED
:107020007A4819680022490800F082FB09B0BDE8DF
:10703000F08F002840F08580BEF1000F14BF0F22B2
:10704000F02201EA020114BF402204221143F1544C
:107050003A78DDE7002800F0B680BEF1000F14BFDB
:107060000F22F02201EA020114BF302003203A78F7
:107070000143F154002ACBD0D8F800E09EF800304C
:10708000A34200F0BA800EF10801002301339342BD
:107090008C4601F10801BBD01EF83300A042F5D1A7
:1070A000DCF80430002BB3D02046012198473A7811
:1070B000AEE7002847D10446BEF1000F14BF0F22EF
:1070C000F02201EA020108BF20460843F0543A7852
:1070D0009EE7002835D0BEF1000F14BF0F22F0222A
:1070E00001EA020114BF1022012211430DF11F0019
:1070F0000022F15401928DF81FA000F08BFB0121BA
:10710000A4F1200301FA03F30193D9E90023C4F1A8
:107110002000CDE90423019B21FA00F003430193F1
:1071200001FA04F30093DDE90023DDE904011043D3
:10713000194302460B469DF81F00C9E9002300F0E1
:1071400091FB3A7864E720200224B5E7BEF1000FF6
:1071500014BF0F22F02297F800E01140F154BEF165
:10716000000F12D0D8F800100B78A34218BF01F11D
:10717000080304D135E011F83020A24232D00130AA
:1071800070459C4603F10803F5D100230DF11F0063
:1071900003938DF81FA000F03DFB0121A4F1200214
:1071A000C4F1200321FA03F301FA02F21A43A140C9
:1071B00003920291D9E90023DDE9020122EA0000ED
:1071C00023EA0101B5E7BEF1000F14BF0F22F02240
:1071D00001EA020114BF102201221143F1543A784E
:1071E00016E78C46DCF80430002BCED02046002178
:1071F0009847CAE7DFF818900DE7F44650E700BF5C
:10720000982900209C29002090290020B0290020E6
:10721000D029002094290020F0B5092A83B0144613
:1072200002D8072003B0F0BD07460E4601F0FCFE71
:1072300018B901F0A1FE0028F4D11C4A1C4B1D4DC9
:10724000176000211C482E7010221C6004F0F5FC11
:107250001A4B00200021751EC3E90001EDB2F6B102
:10726000032600E01D462BB29DF8064017F83300B8
:10727000134A8DF8046007EBC30304F0FC049B7809
:107280008DF805306FF3820401A98DF8064001F0F6
:10729000D5FE6B1E0028C5D1DBB2002DE2D1094A14
:1072A0000948002100F036FABCE700BF942900200D
:1072B00090290020982900209C290020D029002016
:1072C000056F0200856F0200BCBD020070B5084D5D
:1072D0002B785BB1074E00243368012113F834008A
:1072E00001F088FF2B780134A342F5D8002070BD4F
:1072F000982900209429002070B5114D2B7882B078
:1073000053B1104E0024336813F8340001F0D4FF59
:107310002B780134A342F6D802A8002300F8013DDF
:1073200000F078FA084B9DF8070000240025C3E917
:10733000004500F097FA054800F04AFA02B070BD27
:107340009829002094290020D0290020B02900206D
:1073500000B585B000230390194644F2010001AA4C
:107360000193029300F004F805B05DF804FB00BF40
:1073700010B572B6FFF760FCFFF798F90028FBD153
:10738000104B114C11491C1BE408240444F001006B
:10739000FFF7C2FA0E4B1B68DB0700D500BE44F0B6
:1073A00002000C49FFF7B8FABFF34F8F0A490B4BA5
:1073B000CA6802F4E0621343CB60BFF34F8F00BF93
:1073C000FDE700BF24CA0200FCC90200CCBD0200D8
:1073D000F0ED00E0D8BD020000ED00E00400FA0589
:1073E000D0E90223D1E90201994208BF90422CBFA3
:1073F00001200020704700BF244B1B7813B108B157
:10740000037F0BB9002070472DE9D0430446204884
:1074100000F080FB1F4B2049D3E90023D1E900672E
:1074200012EB000843F10009B94508BFB0454046DA
:10743000494603D218F1807049F10001D4E90223D2
:10744000994208BF90420CD3236903B9237763693B
:10745000A069984723690BB1227F4AB90020BDE893
:10746000D08321460D4801F0A9F90120BDE8D08361
:10747000D4E90201C01841F10001C4E9020121462A
:10748000064801F09BF90120BDE8D083582A00206E
:107490000C230020D8290020E8290020ECBD0200A0
:1074A0002DE9F04F85B0814600F00AFB40B17749E5
:1074B000D1E9002312F1807243F10003C1E90023F6
:1074C0004846002100F016FB714D002840F0D380A3
:1074D0004846012100F00EFB002840F0B28003A9CD
:1074E0006C4800F08DFBE8B1694F6B4E0378012BBF
:1074F00000F08480C0F08A80022B09D1002400E0D3
:107500000477664801F06EF90028F9D10123337041
:1075100003A9604800F0A4FB5E4803A900F070FBDB
:107520000028E3D15D48DFF8688101F061F92B683C
:1075300000284CD073B1D8F80030D0E90201D3E96B
:107540000223994208BF904249D2D8F800301B7FED
:10755000002B4DD1514801F045F904465048D4E97B
:10756000026700F0D7FA4F49484BD1E900ABD3E9A5
:107570000023CDE900AB12EB000A43F1000BDDE97B
:1075800000239B4508BF92455046594603D210F14F
:10759000807041F10001301A67EB0101012871F19F
:1075A00000033FDBB0F5350F1CD2A2683C48002138
:1075B0004FF4960300F0FCF970B10D2836D000238B
:1075C00036482B6001F014F92B680028B2D133B98A
:1075D000484600F0C3F902E02B6873B32C6005B095
:1075E000BDE8F08F2E4800F095FA2F4A0244DDE7FF
:1075F000D8F80010294801F0E1F8ABE741682B68A2
:10760000994217D0254801F0F7F881E743681A7FBF
:10761000002A7FF47DAF01221A7741681F4801F0EC
:10762000CDF875E71E48002100F05AFA2046FFF712
:10763000E3FEC4E700233B606AE7484600F08AF9AE
:10764000CCE71748174C00F065FA104BD3E90067F8
:10765000D4E9002316EB000A47F1000B9B4508BF55
:1076600092455046594603D21AF180704BF1000101
:10767000C4E9000133E72B68002B3FF429AF2868E9
:10768000FFF7BAFE00232B6022E700BFD8290020B5
:10769000E0290020482A0020582A0020ECBD0200E2
:1076A0000C230020E8290020FFFFB40010B5124B86
:1076B0001249186882B0582201900823104800F03F
:1076C00049FA08B102B010BD01A90E480E4A00F0F7
:1076D000E1F804460028F5D10A48012100F0E6F956
:1076E00001210B460748094A00F03CF9084B0122EA
:1076F00020461A7002B010BDE8BD0200F02900203B
:10770000482A00200C230020A1740200FFFF7F0004
:10771000582A00204AB10368A1F10101B1FA81F1B0
:1077200049095A611961002070470720704700BF5E
:10773000037F0BB1002070472DE9F043826183B0D5
:1077400004461F480D4600F0E5F91E4B1E49D3E9DB
:107750000023D1E9006712EB000843F10009B945A5
:1077600008BFB0454046494603D218F1807049F140
:1077700000014219266941F10003C4E902237EB9E0
:1077800001A9124800F0FEF988B100254460057097
:1077900001A90E4800F024FA68B903B0BDE8F083EF
:1077A000256101A9094800F0EDF90028EDD1042078
:1077B00003B0BDE8F083024800F0B0F92846ECE7DA
:1077C0000C230020D8290020E8290020482A002086
:1077D00030B5002583B00446057701A90B4800F0B9
:1077E000D1F978B101234460037001A9074800F082
:1077F000F7F908B903B030BD054800F08FF9284605
:1078000003B030BD042003B030BD00BF482A0020C3
:107810000C230020F0B4EFF3108472B60E4B9A687C
:10782000B2B90E4901259D60D1F880700C4D2E46ED
:107830003D401D60C1F88060D1F884505D604FF01C
:10784000FF33C1F88430027004B962B6F0BC7047EF
:1078500001230370F8E700BFA82C002000E100E03E
:10786000FC06FFBD094B9A6872B168B910B4EFF31A
:10787000108172B6064A1C6814605C685460986097
:1078800001B962B65DF8044B704700BFA82C002018
:1078900000E100E070B5274C4379274E04EBC305A7
:1078A00046F823202D7985BB03680A88C3F808258C
:1078B00005798B786AB2002A33DB02F1604202F567
:1078C00061425B01DBB282F80033027953B2002BD4
:1078D00008DB01215B09194D02F01F0201FA02F2D7
:1078E00045F823204279164B164D44F83200581BB8
:1078F00004EBC204C008012300041349237140F0C3
:107900000300FFF709F8002070BD0D4B0D480F492B
:10791000181AC008000440F00200FEF7FDFF08201E
:1079200070BD0B4A05F00F055B012A44DBB21376EC
:10793000CBE700BF642A0020602A002000E100E0BD
:1079400034CA0200FCC902003CBE020018BE02009C
:10795000FCEC00E0036801221A6070470368012212
:107960005A607047F0B404684FF480358D40C4F815
:10797000085306688C00C6F8485304F5A0740668DE
:10798000A4B20027375182B036590468019601F538
:10799000A87122F07F42019E44F821200268C2F8BB
:1079A000445313B10368C3F8045302B0F0BC7047EA
:1079B0002DE9F04104464FF4803600688E40C0F84F
:1079C00048632068C0F8086320688D004719D0F824
:1079D00004E5D7F84005C7F840E505F5A075ADB258
:1079E00027684FF0000847F8058084B0CEEB000010
:1079F0007F59029720F07F40012822F07F47029AAA
:107A000031D02268D2F80455C2F844637A1B22F0C0
:107A10007F42012A01F5A87136D0226842F8217010
:107A20002268D2F80455E843C3F1FF13384403F544
:107A30007F4320F07F40984203D90D2004B0BDE879
:107A4000F08138B9013742F821702268D2F8043544
:107A50009D42F2D1C2F8446323680020C3F8046356
:107A600004B0BDE8F081104A8DE80A0042F001023E
:107A70004FF480609047226842F805805259039283
:107A8000039A9DE80A00BCE72068074B013740F8DD
:107A9000217043F001034FF4806098472268D2F8C8
:107AA00004359D42C9D1D5E710BE02000268022309
:107AB000C2F8443311B10268C2F80433704700BF02
:107AC0000368D3F8040148B10022C3F8042182B04E
:107AD000D3F804310193019B012002B0704700BF2D
:107AE00002684FF480338B40C2F848330268C2F812
:107AF00008337047890001F5A07189B203685858AE
:107B000038B100225A5082B05B580193019B01208A
:107B100002B070470368D3F804057047027953B286
:107B2000002B09DB5B09403302F01F0201210348EF
:107B300001FA02F240F82320704700BF00E100E0A4
:107B4000024B034A1B681068184700BF602A0020D8
:107B5000642A002099B110B4B2FBF3F403FB14249F
:107B6000A4B21CB109205DF8044B704780E81200F4
:107B700084608281C38120465DF8044B70470E20EB
:107B8000704700BF30B482B050E8013F9DB2C48955
:107B900025448489A54228BF2D1B0489A54202BF24
:107BA000BFF32F8F002207E0C5EA030540E8015428
:107BB000002CE9D14FF001028DF803200193019BC5
:107BC0009DF803200B6002F0FF032AB10B880068C8
:107BD000184402B030BC7047184602B030BC704741
:107BE0000A884B889A4201D00020704750E8012F44
:107BF000C2EA024240E80123002BF7D1012070477E
:107C000030B482B050E8023F1FFAA3F5C488A54201
:107C100002BFBFF32F8F00220DE0C4892544848961
:107C2000A54228BF2D1BC3EA054540E80254002C9D
:107C3000E8D14FF001028DF803200193019B9DF8DC
:107C400003200B6002F0FF032AB14B880068184440
:107C500002B030BC7047184602B030BC704700BF5D
:107C60000A884B889A4201D00020704750E8022FC2
:107C7000C2EA224240E80223002BF7D101207047DC
:107C80004A0901F01F03012100EB8200994000F036
:107C900025B800BF10B4012201F01F044B0902FAFD
:107CA00004F100EB8300C9435DF8044B00F024B8F5
:107CB0004B0901F01F0150F82300C84000F00100FB
:107CC000704700BF00B5024652E8000F0B4642E87D
:107CD000003E9EF0000FF7D15DF804FB00B50246B0
:107CE00052E8003F43EA010042E8000E9EF0000F18
:107CF000F6D15DF804FB00BF00B5024652E8003F34
:107D000003EA010042E8000E9EF0000FF6D15DF894
:107D100004FB00BF00B5024652E8003F03EB010040
:107D200042E8000E9EF0000FF6D15DF804FB00BFA4
:107D300000B5024652E8003FA3EB010042E8000E06
:107D40009EF0000FF6D15DF804FB00BF00B50123E3
:107D500086465EE8002F42EA03004EE8000191F0FB
:107D6000000FF6D15DF804FB00B5002386465EE8FF
:107D7000000F00EA03024EE8002191F0000FF6D157
:107D80005DF804FBB8B130B4416882680468521AE7
:107D9000D2B2531E2160DBB242B101680A685C1E98
:107DA000551C0D601370E3B2FF2BF6D10368002061
:107DB000187130BC70470E20704700BF70B582B09C
:107DC00002AB002503F8015D04461846FFF722FDCB
:107DD000236861681A688A4210D9511E19602168A7
:107DE000A3680E68087912F8015C228AE4689B1B7C
:107DF000DBB2984205FB024538BF0B719DF80700C6
:107E0000FFF730FD284602B070BD00BF30B583B02B
:107E100002AB002203F8012D054618460C46FFF779
:107E2000F9FC2A681368591C1160E9682A8A641AE7
:107E3000B4FBF2F41C709DF80700FFF713FD03B0CC
:107E400030BD00BF826802B9704710B5044643696F
:107E50002168006998470023A36010BD0EB400B5E7
:107E600082B0039929B102AA04AB42F8043D00F0A4
:107E7000A1F802B05DF804EB03B070472DE9F04FB4
:107E8000164683B0B1428A4605469846DDF83090E2
:107E90000D9AC0F08B800B460127B3FBF6F39E4290
:107EA00007F10107F9D9474538BF474612F00103EA
:107EB000019302D1B9F1000F57D1AA68012403E060
:107EC00008F1FF3806FB04F4B8F1010FF8D8BAFB4B
:107ED000F4F39E42F6D9DFF8D88011E02B68501CED
:107EE000A86003F802B0AA686B689A4202D32846D9
:107EF000FFF7A8FFB4FBF6F4C4B1BAFBF4F3AA6829
:107F000018F803B0BBF10A0F04FB13AAE6D12B68E3
:107F1000501C4FF00D01A8609954AA686B689A42F2
:107F2000DCD32846FFF78EFFAA68D7E7019BABB1E9
:107F3000B9F1000F12D0B94510D92024AB682A68D6
:107F4000581CA860D454AA686B689A4209F1FF399A
:107F500007D2B9F1000F01D0B945EFD803B0BDE8A1
:107F6000F08F2846FFF76EFFF3E7930718D420241D
:107F7000B945A2D9AA682868531CAB608454AA6882
:107F80006868824209F1FF3905D2B9F1000F95D036
:107F9000B945F0D892E72846FFF754FFAA68F4E7FE
:107FA000B8F1000F14BF20243024E1E701277AE75D
:107FB00064BE02002DE9F04F0D4685B0002900F0A7
:107FC000B2800C78DFF87CA5064691460135002C7E
:107FD00000F0A580252C40F0A88129464FF000082C
:107FE0000D4611F8013B2D2B00F09981302B00F04C
:107FF00099812B2B00F08B812A2B00F0A681A3F115
:108000003002092A00F2D5816A1C002404EB8404A2
:1080100003EB44042A2BA4F13004154600F09681AA
:108020001378A3F13001092905F10102EED91A46AE
:108030002E2A00F09881002701E015F8012F02F0A8
:10804000FB03682BF9D0253A532A63D8DFE812F0F6
:108050002A01620062006200620062006200620047
:108060006200620062006200620062006200620000
:1080700062006200620062006200620062006200F0
:1080800062006200620062006200620062006200E0
:1080900062006200620062006200620062006200D0
:1080A00062006200620062006200620062006200C0
:1080B00062006200620050016200620062006200C1
:1080C0006200620062006200620062003901D10059
:1080D0006200620062006200D10062006200620021
:1080E000620062006200AC00620062006E0062002A
:1080F0005400620062005001D9F800301A1DC9F81E
:108100000020196800943B46CDF8048030460A22CE
:10811000FFF7B4FE01352C78002C7FF457AF337B8A
:10812000002B40F0A68105B0BDE8F08FD9F80030F3
:108130001A1DC9F8002018F0010F1F6840F03C819B
:10814000002F00F0DF81384603F07FFD8046444574
:1081500015D9A4B14FF0200B00E084B1B2683368A8
:10816000511CB16003F802B0B26873689A4204F11E
:10817000FF3402D33046FFF765FE4445EDD8013F9A
:1081800017F8014F002CC5D00A2CB36800F05081BD
:108190003268591CB160D454B26873689A42EFD304
:1081A0003046FFF74FFEEBE7D9F80020131DC9F862
:1081B0000030B36831681468581C3022B060CA546B
:1081C000B3687268934280F02A813268581C782123
:1081D000B060D154B26873689A4280F02581082358
:1081E000002201922146009330461022FFF746FEFE
:1081F00090E7D9F800301A1DC9F80020D3F800B074
:108200008BEAEB73A3EBEB73092B4FF0010108DD55
:108210008AFB0302DB17C3EBA203092B01F1010167
:10822000F6DCB94238BF394634B1BBF1000F02DB8E
:1082300018F0040F00D0013C18F0020F40F0EB8062
:1082400018F0010F18D1002C00F03D818C4213D999
:108250004FF0200CB2683368501CB06003F802C0C5
:10826000B26873689A4204F1FF3480F02E81002CCA
:1082700000F029818C42EDD8BBF1000FC0F254818F
:1082800018F0040F40F02B8108F00303022B00F0DC
:10829000F6808DE8100159463B4630460A22FFF72A
:1082A000EDFD37E7B3683268581C2521B060D15422
:1082B000B26873689A42FFF42DAF3046FFF7C2FDF3
:1082C00028E7D9F800301A1DC9F800201C78B368D7
:1082D0000A2C00F019813268591CB160D454B2687C
:1082E00073689A42FFF416AF3046FFF7ABFD11E713
:1082F000D9F800301A1DC9F80020196800943B46CF
:10830000CDF8048030461022FFF7B8FD02E70D4695
:1083100011F8013B2D2B48F004087FF467AE48F0BC
:1083200001085DE648F002085AE60A2CB36831D02D
:108330003268591CB160D454B26873689A42FFF431
:10834000EAAE3046FFF77EFDE5E60024D9F80030BE
:108350001A1DC9F800206A781B682E2A1C4405F1F2
:1083600001057FF468AE6A78A2F13003092B05F1AC
:1083700001054FF000073FF662AE07EB870702EBFF
:10838000470715F8012FA2F13003092BA7F1300799
:10839000F3D954E6591C3268B1604FF00D01D15445
:1083A000B36872689342C3D33046FFF74BFDB3689E
:1083B000BEE71A4600243BE6B846C7EB080B18F8A0
:1083C000013B9BB10A2BB16842D03268481CB060B7
:1083D0005354B26873689A42EFD33046FFF732FDC8
:1083E000C7EB080B18F8013B002BEBD15C457FF67F
:1083F00091AE2027B3683268591CB160D754B26877
:1084000073689A4204F1FF3402D33046FFF71AFD35
:108410005C45EFD87EE6002F3FF42EAF10E73046E4
:10842000FFF710FDB368D0E63046FFF70BFDD6E648
:10843000591C3268B1604FF00D01D154B3687268B5
:108440009342FFF4A5AE3046FFF7FCFCB3689FE60D
:10845000481C3268B0604FF00D005054B16872682B
:108460009142B2D330460293FFF7ECFCB168029B15
:10847000ABE7304605B0BDE8F04FFFF7E3BC002F97
:108480007FF407AF002C3BD08C427FF602AF4FF059
:10849000300CB2683368501CB06003F802C0B26898
:1084A00073689A4204F1FF3403D24CB38C42F0D883
:1084B000EFE63046CDF80CC00291FFF7C3FCDDF8C3
:1084C0000CC00299F1E70024D6E63046CDF80CC086
:1084D0000291FFF7B7FCDDF80CC00299C7E6B2685D
:1084E000531CB36033682B209854B26873689A4267
:1084F000FFF4CAAE30460291FFF7A4FC0299C3E62E
:108500000024C6E6B84622E6591C3268B1604FF036
:108510000D01D154B36872689342FFF4DCAE30466B
:10852000FFF790FCB368D6E6B268531CB3603368BB
:108530002D209854B26873689A42CBF1000BFFF477
:10854000A3AED7E767666666FFF71CBC2DE9F0416E
:10855000B0F81080A8F104084144CF1C0646FFF78C
:108560002DFCB7FBF8F7044678B3FFB200250123D2
:10857000013FA0F8068006600571437128D080464F
:1085800009E06379AF4203F101036371C8F80000A9
:10859000066080461CD03046FFF710FC01350028ED
:1085A000EFD16679721E234603D0013082421B68E8
:1085B000FBD81F684EB10025236821460135384697
:1085C0001C46FFF723FCAE42F6D10020BDE8F08147
:1085D0002046BDE8F08100BF04300121FFF79ABBBF
:1085E000F8B5012104460430FFF7A2FBC0B200B188
:1085F000F8BD6679721E234603D0013082421B68A3
:10860000FBD81F68002EF3D00025236821460135D2
:1086100038461C46FFF7FAFBAE42F6D1F8BD00BF64
:108620002DE9F041C68890F805E00EFB06FEAEF19C
:10863000040E02EB030C0446E64503F10400154664
:108640000F46B0FBF6F238BFC3EB0E0506FB120077
:1086500012B1013A2468FCD1321AAA4228BF2A4634
:108660008DB14FF000082044AD1A07EB080104302B
:10867000904403F0D7FAB5422A46246828BF324610
:108680000020002DEFD1BDE8F08100BF2DE9F041C1
:10869000C68890F805E015460EFB06FEAEF1040E06
:1086A00005EB030C1A1DE64504460F46B2FBF6F037
:1086B00038BFC3EB0E0506FB102110B1013824684A
:1086C000FCD1721AAA4228BF2A468DB14FF0000889
:1086D0002144AD1A043107EB0800904403F0A2FADC
:1086E000B5422A46246828BF32460021002DEFD12A
:1086F000BDE8F08141DF7047064A074B10B5002402
:1087000014701C60BFF35F8F0448054900F040F807
:10871000204610BD6C2A0020702A0020742A0020F8
:1087200080BE020000B583B002A8002300F8013D1E
:10873000FFF770F8F1EE103A23F09F03E1EE103AE4
:10874000BFF35F8F0A4B4022C3F884219DF80700D6
:10875000FFF788F803F0AEF828B920BF40BF20BF6C
:1087600003B05DF804FBFFF7C5FF03B05DF804FB41
:1087700000E100E0826800239360826813618268F0
:1087800053618268D3608268536082681360704767
:1087900001600B6843604A68934204BF0023436052
:1087A000704700BF426842B101688B681344436060
:1087B0004A68934204BF00234360704770B5446821
:1087C000064620680D4618B908E02468206828B1DC
:1087D000B368294698470028F7D1206828602560AB
:1087E00070BD00BF4368186808B102681A6070471E
:1087F00043681868704700BF4068036873B19942C6
:1088000003D107E0814204D0034618680028F9D15B
:10881000704718460B680360012070471846704780
:10882000184A30B402F59475AB1ADB1003EBD3731E
:108830005B1002EBC30152F83330984228BF0C465C
:1088400005D311E052F8333098420CD221468B1AEE
:10885000DB1003EBD3735B10914202EBC304F1D83E
:10886000094830BC70470D46984204D904F108020B
:10887000AA42D9D3F4E76068034B002808BF184622
:10888000EFE700BF84C20200ACC30200F0B4A34B08
:108890001B685F1C04BFA24B1B78062B00F03481C1
:1088A0009F4AA04B12781B68062A00F01E819B4B42
:1088B0001B685E1C04BF9A4B1B78062B00F00E81D0
:1088C000974A984B12781B68062A00F0F680934B63
:1088D0001B685D1C04BF924B1B78062B00F0C88000
:1088E0008F4A904B12781B68062A00F0A3808B4BAE
:1088F0001B685C1C21D08C4A062B126826D0062BE4
:108900007CD14FF08043D3F80034DA0740F1038183
:10891000824B4FF080421B686FF00101C2F80014D7
:10892000814A062B126869D1033A022A66D97F4A26
:10893000136843F48063136060E0794B794A1B78D5
:108940001268062B40F0AF80C2F30312033A032AE9
:1089500003D8774B9B5C002B46D04FF08052754B71
:10896000D2F80414C3F82015D2F80814C3F824155B
:10897000D2F80C14C3F82815D2F81014C3F82C152B
:10898000D2F81414C3F83015D2F81814C3F83415FB
:10899000D2F81C14C3F84015D2F82014C3F84415BB
:1089A000D2F82414C3F84815D2F82814C3F84C158B
:1089B000D2F82C14C3F85015D2F83014C3F854155B
:1089C000D2F83414C3F86015D2F83814C3F864151B
:1089D000D2F83C14C3F86815D2F84014C3F86C15EB
:1089E000D2F84424C3F870254C4B1B68581C49D05E
:1089F000062B4BD04C4A062B126895D04E4AD2F823
:108A0000883043F47003C2F88830BFF34F8FBFF350
:108A10006F8F4FF01023D3F80022002AC0F2B680E7
:108A2000D3F80432002BC0F2B180444B444A1A60A0
:108A3000F0BC7047C3F30313033B032B3FF657AF60
:108A4000404AD25C12B1404A032111603F4AD35CD4
:108A5000002B3FF44CAF3E4E3E4C3F493F4B052769
:108A6000012500203F223760256008601A603EE73C
:108A70004FF080430022C3F80C21C3F81021C3F843
:108A800038252DE7264B1B78062BB7D1344A234BCC
:108A9000126834491B6802F04F020A60591C7FF4C7
:108AA0002EAF1F4B1B78062BA8D14FF08043D3F875
:108AB0000034DB073FF52CAFA0E7C3F30313033B00
:108AC000032B3FF604AF284AD35C002B3FF4FFAEE4
:108AD000264AD36823F08073D360F8E6244B254AF6
:108AE0001B68C3F342331360EAE6C3F30313033B8B
:108AF000032B3FF6DCAE204AD35C002B3FF4D7AE0D
:108B00001E4B1F4A1A60D2E61E4B1F4A1B68C3F356
:108B100004231360C4E6044B1A6805E73001001013
:108B2000E00F00F0E80F00F0340100103C170040A7
:108B3000D0C3020000C0004000ED00E0142300207C
:108B40000090D003C8C30200A0050040CCC30200BF
:108B500010560040885600401856004014560040F9
:108B600058020010E40E0040C4C30200F0ED00E023
:108B7000440200103C050040C0C3020074C007401E
:108B80000DF0ADBA2403001040350140184B01220E
:108B9000C3F80425D3F80024002AFBD04FF010239B
:108BA00015221349C3F80022D1F80034002BFBD062
:108BB0004FF0102315220E49C3F80422D1F80024E7
:108BC0000B4B002AFAD00022C3F80425D3F8002466
:108BD000002AFBD0BFF34F8F0649074BCA6802F447
:108BE000E0621343CB60BFF34F8F00BFFDE700BFD0
:108BF00000E0014000ED00E00400FA05044B195CC0
:108C00004FF0A04201238B40C2F80C35704700BFE3
:108C1000D4C30200044B195C4FF0A04201238B40E7
:108C2000C2F80835704700BFD4C30200C20770B451
:108C30001AD54FF0A04303224FF400364FF480259D
:108C40004FF400244FF48011C3F84427C3F8482799
:108C5000C3F84C27C3F85027C3F80865C3F8085574
:108C6000C3F80845C3F8081583070AD54FF0A04399
:108C70000C22C3F83427C3F83827C3F83C27C3F8BD
:108C8000402770BC704700BF10B510B101280FD04D
:108C900010BD0E4CA36801226270002BF8D01A6838
:108CA000A2605B6800209847A368002BF7D110BD35
:108CB000064C2369A070002BEAD01A6822615B6819
:108CC000012098472369002BF7D110BD7C2A002092
:108CD00000B1704710B5074CA368012262703BB128
:108CE0001A68A2605B6800209847A368002BF7D140
:108CF00010BD00BF7C2A002030B5012883B027D0EA
:108D00001CD3032818D100F0D9F802A80023264C60
:108D100000F8013DFEF77EFDE368013BE360E36898
:108D200033B9224BD3F8005415B900F0D9F8A57027
:108D30009DF80700FEF796FD03B030BD1C4B0122E5
:108D4000C3F88020BFF34F8FBFF36F8F03B030BDE8
:108D500002A80023144C00F8013DFEF75BFD2378C8
:108D600053B1E3689DF8070001330122E360A2706C
:108D7000FEF778FD03B030BD0E486360A360236149
:108D8000E36000F08DF802F095FD48B1074A012339
:108D90002370D2F80014044A0029E2D09370E0E76F
:108DA00000F08CF8F2E700BF7C2A002000000140B0
:108DB00000E100E0898C020070B50A4A0A4B06788F
:108DC00045688468C06853F8213052F8211084B097
:108DD00003908DF8006001958DF80840684698472B
:108DE00004B070BD942A0020902A002070B50A4A71
:108DF0000A4B067845688468C06853F8213052F8F9
:108E0000211084B003908DF8006001958DF8084022
:108E10006846984704B070BD942A0020902A00202C
:108E2000F0B507460678194D1948DFF870E00C696F
:108E30004B7F45F826400EF8063040F826200C46B9
:108E400094460FCC89B06D460FC594E80F003C786E
:108E50001EF8044085E80F0004965CB9BCF1000FD1
:108E60000C4A07F10C00694608BF002200F0DEFC46
:108E700009B0F0BDBCF1000F074A07F104006946D4
:108E800008BF002200F02EFF09B0F0BD942A002098
:108E9000902A0020ED8D0200B98D0200B42C002034
:108EA000054A13790BB18520704701211060537179
:108EB00018461171704700BF982A0020074B1A68A6
:108EC000D20704D4C02283F8002301221A604FF095
:108ED00080430122C3F81825704700BF00E100E07D
:108EE00010B40B4B0B494FF0804200200224C2F813
:108EF000084383B018601B680193012301980B603D
:108F0000D2F81834DB03FBD403B05DF8044B704790
:108F1000040100400C00004010B5144B1A6882B0E8
:108F200062B10021124A19601B68507900934FF01A
:108F300080410123009CC1F8083390B10D4B1A68A1
:108F40006AB100221A601B6801934FF0804202212F
:108F5000074B0198C2F808131B680120984702B01C
:108F600010BD116853718847E8E700BF0001004059
:108F7000982A00200401004030B5264D95F858305D
:108F800083B013B1082003B030BD6FF02F00401B39
:108F900005F1300305F150044FF0FF31C21821FAFA
:108FA00002F2D20748BF19700133A342F6D14FF045
:108FB000FF33FF240021042217482B606B60AB6055
:108FC000EB602B616B61AB61EB612B6285F850301C
:108FD0006B62AB6285F85230EB6285F8533085F8EE
:108FE000514002F02AFE0D4BC02283F80623402296
:108FF0001A600B4B0B4A002018601B680193019C00
:1090000001214FF0004385F85810C2F8043303B033
:1090100030BD00BFA02A0020F42A002000E100E0BB
:109020007C61004000600040034B93F85800003022
:1090300018BF0120704700BFA02A0020F0B56B4C7C
:10904000231893F93050002D01DB0820F0BD91F872
:1090500002E0CEF3400E9446BEF1000F56D02568D4
:10906000013500F0B480082600256B1C5F4F54F8D2
:109070002320013251D0AB1C9E4245D957F8232002
:1090800001324AD0EB1C9E423ED957F823200132D0
:1090900043D02B1D9E4237D957F8232001323CD0B4
:1090A0006B1D9E4230D957F82370013735D0AB1D68
:1090B000B34229D254F823204C4F01322DD0EB1D5E
:1090C0009E4221D957F82320013226D005F108030A
:1090D0009E4219D957F8232001321ED005F1090309
:1090E0009E4211D957F82320013216D005F10A0308
:1090F0009E4209D957F8237001370ED00B35AE4286
:1091000002D9E36A013307D00420F0BD256A013596
:1091100063D00C260825A8E70B232618DDB244F8F7
:1091200023C086F83050BEF1000F02D1234483F8EB
:1091300048008B785A0715D4DE073FD5830003F12A
:10914000A043D3F8002722F00202C3F80027284FDB
:10915000C60800F0070EBA5D012303FA0EF31343AD
:10916000BB558B78C3F340035BB96AB2083A144429
:10917000097894F8502042EA811284F85020184669
:10918000F0BD6BB29B0003F1804303F5C0430A7846
:10919000D3F8101521F4473121F44071C3F81015AC
:1091A0001204000202F44031D3F8104500F4F852E2
:1091B0000A432243C3F810250020F0BD4A784FF03F
:1091C000A04600F5E073920046F82320BFE7002593
:1091D000C4F800C083F83050ABE7082683F830604D
:1091E0003546C4F820C03346A0E700BFA02A0020BF
:1091F000F42A0020F0B42E4D2E1882B096F83020BC
:1092000053B2072B1CDD2B4493F848309B09032BEA
:1092100040D0012B0CBF4FF400314FF4403180009F
:1092200000F1A040D0F8002722F44032C0F8002717
:10923000D0F800370B43C0F8003702B0F0BC7047DD
:10924000072AFAD8980000F1804000F5C04003F1E9
:1092500040029200D0F8104592B202F180420027FD
:1092600044F0010402F5C042C0F81045019701988E
:1092700017600029E1D096F9302055F82220002A05
:10928000DBD001220B4902FA03F3C1F8043302B028
:10929000F0BC70474FF0A043D3F81035C34013F033
:1092A000010F14BF4FF440314FF40031B7E700BF56
:1092B000A02A002000600040154B034493F83020A2
:1092C00053B2072B16DC072A13D810B49A0002F108
:1092D000804202F5C0420F4CD2F81005012120F067
:1092E000010001FA03F3C2F81005C4F808335DF871
:1092F000044B7047800000F1A040D0F8003723F401
:109300004033C0F80037D0F80037C0F80037704756
:10931000A02A0020006000404FF0A043D3F8103591
:1093200023FA00F000F00100704700BF2DE9F04380
:1093300085B000269F4B01961A68012A47D09E4BA4
:109340001A68012A53D09D4B1A68012A5FD09C4BA2
:109350001A68012A6BD09B4B1A68012A77D09A4B66
:109360001A68012A00F08480984B1A68012A00F0DC
:109370009180974B1A68012A00F09E80954B1A68DD
:10938000012A00F0AB8016F0FF0F1AD0924F012592
:109390000024A30003F18043354203F5C0434FEAA4
:1093A00045050BD0D3F8100557F82420D3F8101535
:1093B000C0F30420C1F3014102B190470134082CED
:1093C000E7D1002EC0F29B8005B0BDE8F083834951
:1093D000D1F8041311F0010100F08F801E601B68AA
:1093E0000293029B744B16461A68012AABD17B4A42
:1093F000D2F804239207A6D500221A601B680293B4
:10940000029B6E4B1A68012A46F002069FD1734AEE
:10941000D2F8042357079AD500221A601B680293DA
:10942000029B674B1A68012A46F0040693D16B4AE7
:10943000D2F8042315078ED500221A601B68029308
:10944000029B604B1A68012A46F0080687D1634ADE
:10945000D2F80423D40682D500221A601B68029336
:10946000029B594B1A68012A46F010067FF47CAF24
:109470005A4AD2F8042390067FF576AF00221A608C
:109480001B680293029B514B1A68012A46F0200682
:109490007FF46FAF514AD2F8042351067FF569AFCC
:1094A00000221A601B680293029B494B1A68012A2A
:1094B00046F040067FF462AF484AD2F80423120611
:1094C0007FF55CAF00221A601B680293029B414B40
:1094D0001A68012A46F080067FF455AF00221A6010
:1094E0001B6803934FF0A043039AD3F82025019201
:1094F00046F00046C3F8202545E70E461FE7384EE4
:10950000A6F15307374C01254FF0A04814F8011F6E
:10951000FF2938D0C9B204AB21F0C00003EBD00260
:1095200001F0070312F80C2C05FA03F31A422AD0B3
:10953000830003F1A04305FA00FCD3F80097D3F8A9
:10954000002722F4403EC3F800E7C9F30142D3F8F4
:1095500000E7022A0CBF4FF440394FF4003949EAC2
:109560000E0907EB000EC3F80097C8F820C59EF956
:10957000303057F8233089092BB1032914D0022A3F
:1095800014D0032A0ED0B442C0D14FF0A043D3F878
:1095900020250192C3F82025019B002BB2D105B0F4
:1095A000BDE8F0830229EED19847ECE70129EAD122
:1095B0009847E8E70061004004610040086100400E
:1095C0000C610040106100401461004018610040CF
:1095D0001C6100407C610040A02A00200060004027
:1095E000F32A0020EF2A0020014B1B68184700BF18
:1095F000FC2A0020104B984201D00020704730B563
:1096000083B002A8002300F8013D0D46FEF702F9E1
:109610000A4B1C7934B19DF80700FEF723F911209D
:1096200003B030BD01229DF807001D601A71FEF7DE
:1096300019F9204603B030BD00200040FC2A00206C
:10964000044B984200D07047034B00221A601A71F5
:10965000704700BF00200040FC2A002030B5714A4E
:10966000D2F8043399058BB05CD5D2F82431002BA5
:1096700058D00023C2F82431D2F8243101934FF49A
:109680000171694B0198C2F8081393F8291009B9C0
:1096900001215160634902228DF81820D1F88024FD
:1096A000C1F880249869D96809920022089007912E
:1096B0009A6193E81200DA6106A8A047594AD2F8E5
:1096C0001C31C3B1584B5869196A884267D993F85D
:1096D000281001F0FF00002961D1C2F81C01D2F866
:1096E0001C11039103999C68186A196A205C013166
:1096F0001962C2F81C054B4AD2F8443183B10021EB
:10970000494BC2F84411D2F8440193F82910009053
:10971000009809B1012111609A69434B002A56D182
:109720000BB030BD3F4AD2F804335B07C6D5D2F840
:109730000831002BC2D03C4B9969002956D000213A
:10974000C2F80811D2F8081104910499D868596A2E
:10975000D2F8182542545A6A996901325A62586AF5
:10976000314A8842AAD1D169002948D192F82920EA
:1097700012B92C4A012151602A4A4FF40171C2F8F2
:109780000813596ADA6808910024012007928DF8BD
:10979000180093E806009C6106A890478EE7214ACE
:1097A00021480021C2F81C11D2F81C210292029A11
:1097B0005B69002B9FD0426983688DF81810416166
:1097C0000793089290E80A0006A8984793E70022BA
:1097D000586AD9689A610122089007918DF818207B
:1097E00006A893E8060090470BB030BDC2F80811F8
:1097F000D2F8080105900598D2F81825AFE7D5688A
:10980000546A1069916100230121D060D3615362D1
:109810008DF818100795089492E80A0006A8984752
:109820004CE700BF00200040042B00202DE9F04150
:109830005F4E05792C2303FB056382B093F82A3031
:109840001BB1082002B0BDE8F0810F46044659491B
:1098500000689046FFF7CEFE18B1112002B0BDE8B7
:10986000F0813A68511C0BD04FF0A0410123934086
:10987000C1F808353B6803F5E073032241F8232063
:109880007B685A1C06D003F5E0734FF0A04200211C
:1098900042F823102368BA69C3F82425397D7B7DFB
:1098A00022680B43C2F86C3597E806002368C3F8BA
:1098B0001425C3F80C153B7D012B4ED02C2303FB44
:1098C00005F3F218C2F804803A69F250B8F1000FBB
:1098D00030D022683B7F384F0021C2F81C11D2F8EB
:1098E0001CE12268CDF804E0DDF804E0C2F8441180
:1098F000D2F84411226800910099C2F804732168DB
:10990000090B4AB2002A4ADB02F1604202F56142C9
:109910005B01DBB282F8003321680A0B53B2002BE3
:1099200009DB01215B09254F02F01F0201FA02F257
:1099300047F8232021682C2303FB0563002204271A
:109940000126C1F8007503F1180EDA619A6183F8F7
:10995000292083F82A605A6174E7BB68591C06D035
:1099600003F5E0734FF0A042002142F82310FB689A
:109970005A1C0DD001224FF0A04102FA03F3C1F8A6
:109980000835FB6803F5E073032241F82320FB68E8
:109990002268B968C2F80835C2F810158EE7084A7F
:1099A00001F00F015B010A44DBB21376B4E700BF9C
:1099B000042B00205D9602008000020000E100E020
:1099C000FCEC00E0F8B5324E047902682C2303FB6E
:1099D000046300215B68C2F80015ABB103682D4A2F
:1099E000C3F808230368190B4AB2002A0DDB520999
:1099F000203201F01F01284D01238B4045F8223011
:109A0000BFF34F8FBFF36F8F0368D3F80CE5D3F824
:109A10001475D3F80815D3F810554FF0FF32C3F87A
:109A20001425C3F80C2503689645C3F80825C3F828
:109A3000102506D00EF5E07E4FF0A043022243F839
:109A40002E207B1C06D007F5E0774FF0A0430222C2
:109A500043F827206A1C06D005F5E0754FF0A043B7
:109A6000022243F825204B1C06D001F5E0714FF08F
:109A7000A043022243F821200068FFF7E1FD2C23D8
:109A800003FB0464002384F82A306360F8BD00BF40
:109A9000042B00208402020000E100E02DE9F041E7
:109AA000344F06792C2303FB067384B05C6903F101
:109AB00010051CB1112004B0BDE8F0815A61996015
:109AC0001C6283F828400268C2F81C41D2F81C11BD
:109AD0000191019A0268012191600268D3F808C0DF
:109AE000C2F81C41D2F81C1102910299D3F82080CF
:109AF000196AD3F804E01CF8088001311962C2F831
:109B00001C85BEF1000F03D0204604B0BDE8F081F3
:109B10005C691A6A0168944288BF754603D819E0E7
:109B200093F828201ABBD1F81C21002AF8D0C1F8DC
:109B30001C51D1F81C210392039AD3F820E01A6A31
:109B40001CF80EE001321A62C1F81CE51A6A944250
:109B5000E9D80168D1F81C31002BFBD00123CB6080
:109B600000202C2303FB067300225A61A3E70F2079
:109B7000F7E700BF042B0020F0B5584BD3F82421A1
:109B80008BB0002A65D1D3F8101100292FD1534B87
:109B9000D3F8442152B10021514AC3F84411D3F8FB
:109BA000444190690394039C00287BD14B4BD3F82C
:109BB000202162B10021C3F82011D3F820210292A4
:109BC0000120474A029CD860506900285DD1434B70
:109BD000D3F858214AB10021C3F85811D3F85801DD
:109BE0003F4A01900198506928BB0BB0F0BDC3F803
:109BF0001021D3F810113A48059105998469D3F8DA
:109C00003C15A142C3D1C469002C5AD0D3F80072CC
:109C1000846127F02004C6680569C3F80042012466
:109C2000C2610891C5600168436807968DF81840C5
:109C300006A89847ABE7D3F84C05936808908DF8D1
:109C400018105161079306A892E80A0098470BB0D4
:109C5000F0BD0021C3F82411D3F82421049202227C
:109C60008DF81820049AD3F880041D4AC3F88004A4
:109C70000990D3F83C05D36808909161D1610793AE
:109C80001168536806A8984781E7D3F84C05936894
:109C900008908DF818105161079306A892E80A0001
:109CA000984794E7D3F83C35D06808930123916135
:109CB000D16107908DF8183006A892E80A009847FD
:109CC00074E7C2688461012308918DF81830079207
:109CD00090E80A0006A8984759E700BF0020004016
:109CE000302B00202DE9F0430479734EE7003B1937
:109CF00006EB830387B093F820301BB1082007B030
:109D0000BDE8F083894605466C4900689046FFF738
:109D100071FC18B1112007B0BDE8F083D9F800201C
:109D2000511C0CD04FF0A04101239340C1F80835DD
:109D3000D9F8003003F5E073032241F82320D9F865
:109D400004305A1C06D003F5E0734FF0A042002106
:109D500042F823102B68D9F81820C3F8242599F865
:109D6000141099F815202B680A43C3F86C252A684B
:109D7000D9F80030D9F80410C2F80C35C2F814151F
:109D800099F81430012B67D03A199200B318C3F830
:109D90000480D9F81030B350B8F1000F4DD02968C5
:109DA00099F81C30DFF81CE10022C1F81021D1F82D
:109DB00010C12968CDF814C0DDF814C0C1F8202105
:109DC000D1F820C12968CDF810C0DDF810C0C1F865
:109DD0002421D1F824C12968CDF80CC0DDF80CC0CD
:109DE000C1F84421D1F844C12968CDF808C0DDF894
:109DF00008C0C1F85821D1F858112A680191019979
:109E0000C2F804E32968090B4AB2002A4BDB02F1CD
:109E1000604202F561425B01DBB282F800332A68DE
:109E2000110B4BB2002B09DBDFF89CE001F01F01A6
:109E30005B0901228A404EF823202A683C4406EB45
:109E40008404002301270825C2F8005584F82070F7
:109E5000E361A361636152E7D9F80830591C06D069
:109E600003F5E0734FF0A042002142F82310D9F827
:109E70000C305A1C0FD001224FF0A04102FA03F31C
:109E8000C1F80835D9F80C3003F5E073032241F826
:109E90002320D9F80C302A68D9F80810C2F8083500
:109EA000C2F8101570E7064A01F00F015B010A4481
:109EB000DBB21376B3E700BF302B0020799B0200A2
:109EC000FCEC00E01003420000E100E02DE9F0416D
:109ED00005794A4C0268EE00731904EB830382B0E3
:109EE0005B68B3B1464BC2F8083303681B0B59B229
:109EF00000290EDB490920310127DFF808E103F0D2
:109F00001F0307FA03F34EF82130BFF34F8FBFF35F
:109F10006F8F711904EB8101D2F80032896923F047
:109F20002003C2F8003241B10023C2F84431D2F814
:109F3000443100930123009953600023C2F8583143
:109F4000D2F8583101937319012104EB8303019F67
:109F5000D1609969D2F85831002BFBD019B1D2F8F1
:109F60004431002BF6D00023C2F8003503684FF0CF
:109F7000FF31D3F80C85D3F814C5D3F80875D3F89E
:109F800010E5C3F80C15C3F8141503688845C3F829
:109F90000815C3F8101506D008F5E0784FF0A04377
:109FA000022143F82810BCF1FF3F06D00CF5E07CFD
:109FB0004FF0A043022143F82C10BEF1FF3F06D022
:109FC0000EF5E07E4FF0A043022143F82E107B1CDB
:109FD00006D007F5E0774FF0A043022143F82710A1
:109FE0001046FFF72DFB354404EB8504002384F86D
:109FF0002030636002B0BDE8F08100BF302B00204C
:10A000001003420000E100E0F0B501F06043B3F15D
:10A01000005F83B0047902D0102003B0F0BD4FEA96
:10A02000C40E234F0EEB040507EB85056B6913B1D6
:10A03000112003B0F0BD6A61A9600268C2F8203146
:10A04000D2F820C10268CDF800C0DDF800C0C2F827
:10A050005831D2F8582101920268DDF804C06E69C7
:10A06000C2F84415C2F848650268012191606A6827
:10A070000AB11846D1E7036800E0BAB9D3F8201155
:10A08000D3F85821003218BF01220029F5D06AB94F
:10A090000122DA600268D2F85831002BFBD0002090
:10A0A000744407EB840400226261B6E70F20F7E7EF
:10A0B000302B002072DF704773DF704776DF704708
:10A0C0007ADF70477CDF70477FDF70478FDF704734
:10A0D000B1DF7047FDF73CB9FDF73AB908B5037831
:10A0E00003B108BD054B3B211888FFF7E7FF0028A7
:10A0F000F7D0BDE80840FDF72BB900BF20230020B2
:10A100000D2820D1114B1248181AC008000410B5B0
:10A1100040F003000C460F49FCF7FEFB0E4B0F49C5
:10A120001888224601F01EFB30F008020DD043F2E1
:10A130000202904209D043F20142904205D0BDE8AC
:10A140001040FDF705B9FDF703B910BD24CA0200A0
:10A15000FCC9020004C4020020230020542B00206C
:10A1600008B502206AB9FEF755FD094B09480A49AE
:10A17000181AC008000440F00300BDE80840FCF7CE
:10A18000CBBBFEF73BFD024B02480449F0E700BFA2
:10A1900024CA0200FCC9020034C4020020C4020028
:10A1A00010B50388103B82B00446462B46D8DFE842
:10A1B00003F06724458345454545454545454545A7
:10A1C0004545455145454545454545454545454533
:10A1D000454545454545454545454545454745452D
:10A1E000454545454545454545454545454545451F
:10A1F000454545455D4545454700364B3648374959
:10A20000181AC008000440F00300FCF785FB012089
:10A21000FEF700FD324B4FF6FF721A80FDF76CF827
:10A2200008B1FDF795F82F4B01211878FFF744FF8F
:10A2300008B1FDF78DF80020FEF7E0FC02B010BD7C
:10A2400080881321FFF73AFF0028F7D0FDF780F848
:10A2500002B010BD002380888DF8043001A98DF86C
:10A260000530FFF733FF0028E8D0EFE71C4B002153
:10A2700018880A460B46FFF72BFF0028DED0E5E7DB
:10A28000144B15481849181AC008000440F0030080
:10A29000FCF742FB0120FEF7B1FC0020FEF7BAFC00
:10A2A0000F4BA1881148198001F05AF970B9FDF7D8
:10A2B0000DF80028C2D0C9E7094B00221888852173
:10A2C0001346FFF701FF0028B8D0BFE7FDF740F8BD
:10A2D000EDE700BF24CA0200FCC9020054C402001A
:10A2E000202300202223002048C40200A02B0020AD
:10A2F00080B50020A6B04FF48041FCF783F908B187
:10A30000FDF726F8FCF70CF90120FEF78FFCFDF7AE
:10A31000CDF908B1FDF71CF87848012140F233323D
:10A32000FCF77AFF08B1FDF713F8FEF7E5F908B17D
:10A33000FDF70EF801F038FA08B1FDF709F826AC80
:10A34000002344F83C3D0120214601F001FB08B107
:10A35000FCF7FEFF204601F0B5FB08B1FCF7F8FF63
:10A360009DF820306648012262F3030326AD62F3B4
:10A37000071305F8783D01F068FC614982B2284670
:10A38000FFF7A0FE08B1FCF7E3FF002108222046FA
:10A3900001F053FC5026A02100224FF4C873204640
:10A3A000ADF85C60ADF85E10ADF86020ADF86230DD
:10A3B000FFF786FE08B1FCF7CBFF5248002100F002
:10A3C00071FF08B1FCF7C4FF00224F4B4F480892C1
:10A3D0002146179301F0B2F808B1FCF7B9FF4C4BD6
:10A3E0004C480893294601F055F908B1FCF7B0FF35
:10A3F000484B494E9B7C8DF80630002141F2235397
:10A400003C222846ADF80430012701F016FC062353
:10A410004FF0020E00213C2220468DF823308DF8AB
:10A4200020E08DF8227001F008FC324601AB28468E
:10A4300052F8041BADF86C701C9300F0E5F808B1FD
:10A44000FCF786FFB168354A204600F0DDF808B118
:10A45000FCF77EFF0021182202A801F0EEFB012587
:10A460000023402602AA2E482B498DF81D508DF856
:10A470000850ADF8143003938DF81C300496FFF7A4
:10A4800019FE08B1FCF764FF204600211C2201F0F0
:10A49000D4FB4FF4A026002320464FF4A03503241C
:10A4A0002049214A1793ADF86A308DF86C30189620
:10A4B00019958DF868401C911D9200F0F7FB08B1CA
:10A4C000FCF746FF194B1A481A49181AC00800042D
:10A4D00040F00300FCF720FA114B01211878FFF738
:10A4E000EBFD08B1FCF734FF0020FEF787FBFCF71B
:10A4F000DDF80028FBD1FEF715F9F8E71823002056
:10A5000064C402008C2B0020D5A00200A02B0020E8
:10A5100061A10200542B00202423002030230020BE
:10A5200022230020DDA00200D9A0020024CA0200DC
:10A53000FCC9020074C402006DDF704779DF704708
:10A540007DDF704764DF70472DE9F04F85B08346AB
:10A550000E9D00882C880194BDF83C9000284ED0B8
:10A5600000278A46164698463C4604E0BBF8003071
:10A570000134A34226DDDBF8043053F824000390B5
:10A580000DF10B0103A80022FFF7DCFF18BB9DF8BB
:10A590000B30B342EAD10FB32A8893194B4519DC2B
:10A5A000424403A80DF10B010127FFF7CBFF90B93F
:10A5B0002B889DF80B2013442B80BBF8003001340E
:10A5C000A342D8DCDFB12B88019A013B9B1A9BB2D6
:10A5D000FF2B12D90C2005B0BDE8F08F2B885A1C38
:10A5E000334402334B4592B2F4DC2A8008F802A0CF
:10A5F0002A88013292B22A80D2E708F8023000207D
:10A6000005B0BDE8F08F00BF2DE9F04700231788A3
:10A61000138090F82D3084B0144605460E46002B6A
:10A6200040F00281AA78002A40F02A81EA78002AC4
:10A630002CD1696899B1DA1CBA42097822D8022271
:10A64000F254238801339BB20A222380F2542388D8
:10A6500001339BB22380F1542388013323802B895B
:10A66000002B40F033812B8A002B40F048812B8B4C
:10A67000002B40F05D81296A00295CD023889A1D57
:10A68000BA4218D90C2004B0BDE8F087D91CB942F1
:10A69000F8D80221F154238801339BB20121238091
:10A6A000F15423880B449BB22380F25423880B443B
:10A6B0009BB22380BDE70A88052A40F203816FF42C
:10A6C000486802EB080080B24FF27D3E704540F2D0
:10A6D000F9804888052840F2F5806FF4486C84447E
:10A6E0001FFA8CFCF44540F2ED804FF6FF7E724578
:10A6F00004D0704502D0824200F2E4800522F25478
:10A70000238801339BB212222380F2542388013321
:10A710009BB223800A88F2543344120A5A70238869
:10A7200002339BB223804A88F2543344120A5A708F
:10A73000238802332380D5F82480B8F1000F2FD06E
:10A74000B8F804202188131D0B44BB429AD8931CEF
:10A75000FE2B97D803327254238801339BB2FF2219
:10A760002380F254238801339BB22380B8F8002061
:10A77000F2543344120A5A702088023080B220808A
:10A78000B8F8042062B1D8F80810002900F09A80C7
:10A79000304401F047FAB8F804302288134423808B
:10A7A00095F82C30002B40F0DC80287800283FF40E
:10A7B0006AAF2B88012B00F0858023889A1CBA424F
:10A7C0003FF660AF012805D16978023119448F4204
:10A7D000FFF458AF023FFB1A04A99FB221F8087D8D
:10A7E000B018FFF7ADFE00287FF44DAF2A78022A9B
:10A7F00000F008816978BDF808309942C0F0FD800A
:10A800009F42C0F0FA800921FE2B3FF63BAF228821
:10A810005D1CB5542288013292B22280B154228844
:10A820000132134423802EE7082F7FF62BAF02A8B6
:10A83000FFF782FE00287FF426AF23880822F25417
:10A84000238801339BB21B222380F25420880130DD
:10A8500080B22080062230440DF1090101F0E2F9B6
:10A8600023889DF8082006339BB212F0FE0218BF21
:10A8700001222380F254238801339BB22380D1E646
:10A880000433BB423FF6FEAE02A8FFF757FE002896
:10A890007FF4F9AE2388BDF808200321F154238802
:10A8A00001339BB219212380F154238801339BB2D9
:10A8B000F1182380100AF2544870238802339BB2A7
:10A8C0002380B3E6072004B0BDE8F08705F108084F
:10A8D00002218DE8900040460A463346FFF734FED9
:10A8E00000287FF4D0AE8DE890004046062110226B
:10A8F0003346FFF729FE00287FF4C5AEB3E605F125
:10A9000010088DE890004046032102223346FFF7ED
:10A910001BFE00287FF4B7AE8DE89000404607216B
:10A9200010223346FFF710FE00287FF4ACAE9EE6FF
:10A9300005F118088DE890004046142102223346A4
:10A94000FFF702FE00287FF49EAE8DE8900040469F
:10A95000152110223346FFF7F7FD00287FF493AE50
:10A9600089E6D5F82880B8F1000FABD0B8F80420FC
:10A970000232FE2A3FF686AE23884FF000094FF0E0
:10A98000160A0132F254238801339BB2238006F861
:10A9900003A0238801339BB22380B8F80020F2542F
:10A9A0003344120A5A70238802339BB22380B8F8CA
:10A9B0000410F0180A4661B1D8F808301946002B87
:10A9C00080D001F02FF9B8F80430228813449BB2EC
:10A9D000238009F1010995F82C205FFA89F94A458D
:10A9E00009EB49087FF6E1AEAA6A02EB8808B8F8DD
:10A9F00004200232FE2AC4D944E6012A08D03B468C
:10AA0000082101E7BDF808309F42BFF4FCAEF6E72D
:10AA10008F42F4D30B460821F6E600BF75DF70477E
:10AA200076DF70477ADF70477BDF704770B51D4C6B
:10AA3000238885B2AB4282B001D002B070BD1A4EFD
:10AA4000217A327B91420FD3337C00222272BBB930
:10AA50007369002BF1D00022ADF806508DF8042068
:10AA600001A8984702B070BD184604F10A01FFF72B
:10AA7000D5FF88B11128E0D0B369002BF1D1DCE714
:10AA800028463B21FFF7CCFF30F00803E0D0B36944
:10AA9000002BDDD09847DBE7237A0133237202B025
:10AAA00070BD00BFE82B0020CC2B0020F0B5028841
:10AAB000112A83B0034654D040D9122A08D0502A14
:10AAC00004D1774DC188EA8991425CD003B0F0BDD2
:10AAD000744C828821889142F8D1E589268A408980
:10AAE000618940F2F31C65454FF6FF7E05EB0C07CC
:10AAF00094BF6D1BCCEB0505764594BFB61BCEEB22
:10AB00000606814256D8A189814253D399898D4244
:10AB100050D88F424ED3DB899E424BD8604B596947
:10AB200001200023607223720029CFD00123ADF8E9
:10AB300006208DF8043001A88847C7E7102AC5D140
:10AB4000C17B82880129C1D1564C26884FF6FF71FE
:10AB50008E423ED0524B9B69002BB7D004209847C1
:10AB6000B4E7504C828823889A42AFD16068FCF7E2
:10AB70002FFE18B14A4B9B6903B198474FF6FF73FC
:10AB8000238003B0F0BD028A022A9FD1454C8788FA
:10AB90002688BE429AD1123000F07CF9002862D19A
:10ABA0006068FCF715FE002890D0AB69002B8DD0B3
:10ABB00098478BE73A4D267AAB6869686068002E43
:10ABC00018BF194600236372FCF7B2FD0028ECD1D0
:10ABD0007CE7354D228003CDC4F80E10C4F80A007E
:10ABE0006589588AE189B4F810E000278542277208
:10ABF0002AD8A589854227D340F2F31081429D8A45
:10AC000094BF481A081AA8421ED801F2F311A942AB
:10AC10001AD3B645DB8A94BFCEEB0E0EC6EB0E0EF2
:10AC20009E4511D81E4BD8890121617200287FF4FE
:10AC30004DAF5B69002B3FF449AF8DF80410ADF8C0
:10AC4000062001A8984741E7154D1648EB890021D9
:10AC50006172002B7FF43AAF40686968FCF768FDC9
:10AC60000028A2D132E7637A63B96968AB68277AB2
:10AC700060683246002F18BF1946FCF759FD0028BE
:10AC800093D123E76B6900222272002B3FF41EAFA1
:10AC90000122ADF806708DF8042001A8984715E749
:10ACA000CC2B0020E82B0020202C002060B3F8B52E
:10ACB000054606460FCDDFF870E0174F74460FC407
:10ACC000844695E80700CEF8007084E80700BCF1E0
:10ACD000000F1BD06046FFF7A5FEA0B933681868C7
:10ACE000596803C70D4B0E490E4A18464FF6FF74BC
:10ACF00040F8041F1C800021FCF70CFD002814BF45
:10AD000003200020F8BDF8BD0E2070473846FFF73D
:10AD10008BFE0028E6D0F8BD202C0020E82B002078
:10AD2000002C00202DAA0200CC2B00202DE9F04F92
:10AD30000388B0F804A0103B99B081460A2B1BD8B9
:10AD4000DFE803F02F281A1A1A1A1A1A1A1D060019
:10AD5000047A47482409032C51466AD8FCF79AFF25
:10AD6000032C68D043485146FCF794FF022C66D070
:10AD700051464148FCF78EFF19B0BDE8F08F037AC9
:10AD8000002BF9D1437A3A481B0751466DD4FCF7A2
:10AD900081FFF1E751463948FCF77CFF19B0BDE867
:10ADA000F08F374A936818A8DB4340F8603D51683C
:10ADB000FCF7A2FF009B0193019B8BB34FF00008AF
:10ADC000444601A82146FCF773FF30B118AB03EBF2
:10ADD000480308F1010823F8284C0134142CF0D161
:10ADE000CDF834800DAD0FCD02AC0FC40FCD0FC424
:10ADF00095E8070084E80700B8F1000F10D0214E55
:10AE00000DF10A0B00273BF8025F1F4C2046294634
:10AE10000434FCF73FFFB442F8D101374745F2D183
:10AE2000BAF1130F10D90420FCF792FA19B0BDE85B
:10AE3000F08FFCF725FF0F485146FCF721FF5146E4
:10AE40000D48FCF71DFF97E70C485146FCF718FF2B
:10AE50000D485146FCF714FF99F80F30022B8BD1A7
:10AE600051460A48FCF70CFF86E7FCF709FF83E729
:10AE7000402C00203C2C0020382C0020302C0020BE
:10AE8000282C0020A42C00202C2C0020342C002066
:10AE9000AADF7047007800F001007047F0B58B78AA
:10AEA00091B0002B0C460988ADF80C1008BF0123A7
:10AEB000064615466846032200218DF80E3000F044
:10AEC000BCFE9DF80020637C02F0F0026FF30712D5
:10AED000013B8DF80020042B10D8DFE813F020018F
:10AEE0002A010500350116019DF80030012262F3A8
:10AEF0000303032262F307138DF800309DF801204D
:10AF0000A37C02F0F0026FF30712013B8DF80120E1
:10AF1000042B10D8DFE813F02D0137010500EE00F7
:10AF200023019DF80130012262F30303032262F33F
:10AF300007138DF801309DF80230E77B227D207CDD
:10AF4000217B67F3C303002A60F3041314BF0222BA
:10AF5000012261F3000362F3420309A800211C22CD
:10AF60008DF8023000F069FE637B13F0300F40F083
:10AF70008F80627BA37B8DF824200021142204A8FB
:10AF80008DF8253000F059FEA368A288CDF814D0C2
:10AF900003A90491ADF81C201BB1E2880893ADF819
:10AFA0001820A369002B44D001AF002103223846AA
:10AFB00000F043FEA2699DF804101388ADF82C3010
:10AFC0005388ADF82E3050680D97137B0A9001F02E
:10AFD000F0016FF30711013B8DF80410042B3DD8ED
:10AFE000DFE813F01B0125013200F20011019DF88A
:10AFF0000530012161F30303032161F307138DF889
:10B000000530917A9DF8063061F3C3038DF8063060
:10B01000D17A61F304138DF80630117A927B002AFD
:10B0200061F3000314BF0222012262F342038DF890
:10B030000630E36903B10C93304609A904AA2B46F4
:10B04000FFF726FF11B0F0BD9DF80430012161F338
:10B050000303032161F307138DF804309DF80510F5
:10B06000537B01F0F0016FF30711013B8DF80510E0
:10B07000042BC6D801A151F823F000BFF3B10200A0
:10B08000B3B10200EFAF02009DB10200DFB10200D8
:10B09000032202A8002100F0D0FD9DF80920E37CE6
:10B0A00002F0F0026FF30712013B8DF80920042B28
:10B0B0000ED8DFE803F0D1DB03E6C7009DF80930C6
:10B0C000012262F30303032262F307138DF80930B0
:10B0D0009DF808309DF80A1002AA0E92012262F330
:10B0E000030362F3071362F342018DF808308DF811
:10B0F0000A103EE79DF80130022262F303030122A9
:10B1000062F307138DF8013015E79DF80030022235
:10B1100062F3030362F307138DF80030EEE69DF847
:10B120000030012262F3030362F307138DF800304D
:10B13000E4E69DF80030012262F30303022262F389
:10B1400007138DF80030D9E69DF80030022262F333
:10B150000303012262F307138DF80030CEE69DF859
:10B160000130022262F3030362F307138DF801300A
:10B17000E1E69DF80130012262F3030362F3071355
:10B180008DF80130D7E69DF80130012262F3030308
:10B19000022262F307138DF80130CCE69DF80530EA
:10B1A000022161F30303012161F307138DF80530D8
:10B1B00027E79DF80530012161F30303022161F3C4
:10B1C00007138DF805301CE79DF80430022161F368
:10B1D0000303012161F307138DF804303EE79DF866
:10B1E0000530022161F3030361F307138DF8053085
:10B1F00007E79DF80530012161F3030361F30713AD
:10B200008DF80530FDE69DF80430022161F303035B
:10B2100061F307138DF8043020E79DF80430012115
:10B2200061F3030361F307138DF8043016E79DF80B
:10B230000430012161F30303022161F307138DF848
:10B2400004300BE79DF80930022262F3030362F336
:10B2500007138DF809303BE79DF80930012262F3AE
:10B26000030362F307138DF8093031E79DF80930C5
:10B27000012262F30303022262F307138DF80930FF
:10B2800026E79DF80930022262F30303012262F3EC
:10B2900007138DF809301BE790DF7047A5DF704773
:10B2A000B5DF704788B110B417221B240023016159
:10B2B00002804280C28002810471047344738372ED
:10B2C000C3725DF8044B184670470E20704700BFEC
:10B2D00070B5858884B02DBB0388232B0C4600F005
:10B2E000C58021D93A2B00F0B080552B70D0242B8B
:10B2F00000F09780A37AABB10020E188FFF7CEFF82
:10B30000002800F08A8011280CD0FDF789FA824BC2
:10B310008249024682481B1ADB08180440F00100EB
:10B32000FBF764FB04B070BD102B0AD0112BE1D1E8
:10B3300017221B238D72CD72CA800A810B734B7347
:10B34000F0E70B790B73C27B012A00F0B780022A69
:10B3500000F0B180C98822898A42C0F0C080627B37
:10B360009A42C7D200259BB2284602A96A46ADF888
:10B370000830ADF80A30ADF80C50ADF80E5000951D
:10B38000ADF80450FFF788FF0028B3D0624B644E3D
:10B390009E1BF608FDF744FA360446F00106034604
:10B3A0002A4630465F49FBF793FBBDF80020BDF805
:10B3B000023002B91BB130465B49FBF789FBBDF88F
:10B3C0000420002A96D030465849FBF70FFB91E73E
:10B3D000C388C988A572172B38BF17238B4228BF93
:10B3E0000B4628462381FFF75BFF002869D1E37AEB
:10B3F000002B7FF47FAF2269002A3FF47BAF2189C5
:10B40000ADF80A3040F67720ADF80800ADF80C1022
:10B41000204602A99047A37A6DE70122A072E2724A
:10B4200080E70B69027A4A73002B3FF463AF4DF655
:10B430007A210295ADF80C50ADF808108DF80C206B
:10B44000204602A99847A37A55E7E38841892269F3
:10B450008B4228BF0B46172B38BF172323810AB115
:10B46000E17AE1B90023E372A3725BE70B7B027A16
:10B47000ADF80C50934228BF1346284602A96A46ED
:10B48000ADF80E500095ADF80450ADF80830ADF8A9
:10B490000A30FFF701FF00283FF42CAF76E740F6B3
:10B4A0007721ADF80810ADF80A50ADF80C30204601
:10B4B00002A99047D6E74988E1804CE70988E180F6
:10B4C00049E7FDF7ADF9144B1949024614481B1A18
:10B4D000DB08180440F00100FBF788FA87E700203A
:10B4E000FFF7DCFE18B90123E372237B37E711284D
:10B4F00003D10123A372237B31E7FDF791F9064BBA
:10B500000649024606481B1ADB08180440F00100F1
:10B51000FBF76CFA237B22E744CA020070C50200E5
:10B52000FCC902008CC40200D8C4020018C5020085
:10B53000A4C50200B0DF704766DF704770B169B123
:10B540000378DE2B08D00B684360DE224FF6FF73D2
:10B550000270438000207047082070470E2070471B
:10B5600020B10378DE2B03D0082070470E207047EF
:10B5700041800020704700BF19B110B10B78DE2B5D
:10B5800000D07047F0B5054683884888984285B05A
:10B590000C4625D02B88112B40D0512B03D0012BEA
:10B5A0002BD005B0F0BD6688AB88B342F9D1AF7936
:10B5B000022FF6D1AB7B042B3BD0062B39D0052BC9
:10B5C000EFD168460021102200F037FB6D468DF860
:10B5D000007030462946FFF7ADFF0028E1D01AE0A1
:10B5E0000B7A002BD6D00021FFF7A6FF0346F0B15F
:10B5F00011281BD063689847CCE72E7AAB88012EC0
:10B60000CFD160889842CCD126720021FFF794FFF9
:10B61000E0B111281CD063689847C2E7AA88638804
:10B620009A42BED14FF6FF736380BAE701232372BB
:10B63000B0E700234FF4C072009301930293039389
:10B640008DF80070ADF804206D46C2E72072A8E7BF
:10B650002672A6E7A8DF7047AEDF704762DF70474B
:10B660000288502A034600D0704710B44A88DC880C
:10B67000944202D05DF8044B70471A8A012AF9D12E
:10B680004C69002CF6D098889A7C23465DF8044BD0
:10B69000184700BF70B5324C0E68A2686168E36855
:10B6A0008EB0054620686E6102AC0FC405F1120130
:10B6B00002A8FFF7D3FF08B10EB070BD0EA941F28A
:10B6C000235321F8343D0120AB7C8DF806302A4607
:10B6D000FFF7C0FF0028EFD10146202206A800F0A6
:10B6E000ACFA9DF82530A97C8DF81A102A46012461
:10B6F00043F0120341F2245632F80A0B8DF825303C
:10B7000006A9ADF81860ADF81E40ADF81C408DF8E4
:10B7100029408DF82B40FFF7C1FB0028CCD1014612
:10B72000202206A800F089FA2A469DF82530AE7C32
:10B7300032F8020BADF81E4043F00A0341F22555E2
:10B7400006A9ADF81C408DF829408DF82A408DF8E7
:10B750001A608DF82530ADF81850FFF79FFBABE766
:10B76000E4C5020070B588B00E4605468DF8072086
:10B77000012404A800211022ADF80E4000F05DFA6B
:10B780007389ADF810300DF107020DF10E03284654
:10B7900004A98DF8124007920693FFF75DFF08B0E9
:10B7A00070BD00BF10DF704770B5394D2B7884B085
:10B7B00013B1082004B070BD364E3749012302A8EA
:10B7C0003370FCF7E5FF039B5BB11A6859680020F2
:10B7D00090470028EED002A8FCF7E4FF039B002B63
:10B7E000F3D102A82D49FCF7D3FF039B4BB11A6894
:10B7F00059680020904702A8FCF7D4FF039B002B58
:10B80000F5D1274B18680190002302A88DF8083065
:10B81000FCF700F801A82349FFF7C4FF0446B0FA7B
:10B8200080F39DF808005B092B70FCF71BF80CB146
:10B830002046BFE71C4B1D491C70347091F816233D
:10B84000EC2352091341DB0717D5194B9A68CAB983
:10B850004FF480030B6002A81049FCF799FF039B8B
:10B860004BB11A6859680120904702A8FCF79AFF6B
:10B87000039B002BF5D100209CE742F20200FBF76E
:10B8800067FDE8E71A6842F480021A60E3E700BF48
:10B89000A42C0020A52C0020F8C5020004C602003C
:10B8A000F4C5020071730200A62C002000E100E044
:10B8B000A82C0020014B1878704700BFA42C002052
:10B8C00000B583B068460849FCF762FF019B43B1AD
:10B8D00058681A6890476846FCF764FF019B002B84
:10B8E000F6D103B05DF804FB18C6020060DF7047B4
:10B8F00069DF704761DF7047134B1B7813B310B5D6
:10B90000342490B003A80DF10201ADF80240FFF716
:10B91000F1FF88B901A80D49FCF73AFF029B002B03
:10B92000F0D01A68596803A8904701A8FCF73AFFBD
:10B93000029B002BF5D1E5E7052801D0FBF708FDB8
:10B9400010B010BD704700BFA72C002024C6020015
:10B9500070B50C4684B0002978D0524B0B60054678
:10B9600000210C2201A800F068F90126062301A994
:10B97000202022688DF804508DF80660ADF808305C
:10B98000FFF7B6FF002864D100210C2201A800F0C7
:10B9900054F901250023402001A922688DF80550A3
:10B9A0008DF806308DF80730FFF7A2FF002830D160
:10B9B00000210C2201A800F040F90A23012001A96E
:10B9C00022688DF80430FFF793FF00285CD1002136
:10B9D0000C2201A800F031F94FF4B063A12001A9B5
:10B9E00022680193FFF784FF00283FD100210C2239
:10B9F00001A800F022F99DF8043022686FF30003DB
:10BA000001A9A0208DF80430FFF772FF70B904B0CF
:10BA100070BDFCF705FF244B2449024624481B1A3D
:10BA2000DB0818042843FAF7E1FFC1E7FCF7F8FE4A
:10BA30001D4B204902461E481B1ADB08180440F023
:10BA40000100FAF7D3FF002004B070BD0E2004B04F
:10BA500070BDFCF7E5FE144B1749024614481B1A4B
:10BA6000DB0818043043FAF7C1FF8DE7FCF7D8FE76
:10BA70000D4B124902460E481B1ADB08180440F011
:10BA80000100FAF7B3FFB1E7FCF7CAFE064B0C4919
:10BA9000024607481B1ADB08180440F00100FAF7B9
:10BAA000A5FF94E7F022002054CA020078C60200E5
:10BAB000FCC9020064C7020030C6020010C70200C1
:10BAC000C4C60200F8B504460768FFF70FFF2368F5
:10BAD0009F42064605D326BB1A4B01221A703046F8
:10BAE000F8BD194B194D1A495D1BED082D0445F0A1
:10BAF00002052846FAF710FF28463A4615492368FA
:10BB0000FAF7E6FF4FF080532268D3F80C31124960
:10BB10009B0203F1005328469A1AFAF767FF002E9A
:10BB2000DAD03046FCF77CFE074B0C49024607484A
:10BB30001B1ADB08180440F00100FAF757FF3046E3
:10BB4000F8BD00BFA72C002054CA0200FCC90200A7
:10BB5000B8C70200E8C702001CC8020048C80200BB
:10BB60004BDF704700B585B001A8FFF7F9FFA8B912
:10BB700002A80E49FCF70CFE039B002BF4D01A68B8
:10BB800059680198904702A8FCF70CFE039B002B14
:10BB9000F5D101A8FFF7E4FF0028E9D0052801D07E
:10BBA000FBF7D6FB05B05DF804FB00BF74C80200CC
:10BBB00008B5074B044613B10021AFF30080054BD5
:10BBC0001868836A03B19847204600F047F800BF21
:10BBD0000000000090C9020070B50E4B0E4CE41A34
:10BBE000A41000251E46A54204D056F825309847DB
:10BBF0000135F8E700F034F8084C094BE41AA410BA
:10BC000000251E46A54204D056F825309847013538
:10BC1000F8E770BD98230020982300209C23002083
:10BC20009823002010B5431E0A44914204D011F815
:10BC3000014B03F8014FF8E710BD0244034693425D
:10BC400002D003F8011BFAE77047034613F8012BF3
:10BC5000002AFBD1181A013870470000FEE700BF28
:10BC6000F8B500BFF8BC08BC9E467047F8B500BFE9
:10BC7000F8BC08BC9E467047FFFFFFFFFFFFFFFFB9
:10BC8000FFFFFFFFFFFFFFFF0000000000000000BC
:10BC90000000D60106010000F563020061640200A5
:10BCA000F1630200756172745F6C6F675F6261635C
:10BCB0006B656E64000000004261636B656E6473C7
:10BCC00020666C7573686564000000006170700028
:10BCD000E82800207F0000007829002000000000F4
:10BCE0009CBD0200A4BD0200ACBD0200B4BD0200B8
:10BCF00034BD020064BD02002CBD02006CBD020018
:10BD000074BD02007CBD020084BD02008CBD020037
:10BD100094BD020025734C6F67732064726F70705E
:10BD20006564202825642925730D0A001B5B313BBF
:10BD300033316D001B5B306D000000002573000087
:10BD40003C25733E2025733A200000000D0A0000B8
:10BD50002025303278000000202020007C000000E8
:10BD6000256300001B5B313B33306D001B5B313BB7
:10BD700033326D001B5B313B33336D001B5B313B5A
:10BD800033346D001B5B313B33356D001B5B313B46
:10BD900033366D001B5B313B33376D006572726F5C
:10BDA000720000007761726E696E6700696E666F7F
:10BDB000000000006465627567000000B029002083
:10BDC0006170705F627574746F6E000046617461BB
:10BDD0006C206572726F720053797374656D207296
:10BDE000657365740000000001000600000000009B
:10BDF0005C2A0020E17302006170705F74696D65F8
:10BE000072000000000000000000000000000000C0
:10BE10000338FDD87047000052544320696E737494
:10BE2000616E636520616C726561647920696E6919
:10BE30007469616C697A65642E0000005254433A5B
:10BE400020696E697469616C697A65642E0000000E
:10BE50005254433A20556E696E697469616C697A0F
:10BE600065642E003031323334353637383941424B
:10BE7000434445467077725F6D676D740000000043
:10BE8000A0C90200A0C9020004000000736F727410
:10BE90006C697374000000004E52465F5355434373
:10BEA000455353004E52465F4552524F525F5356D0
:10BEB000435F48414E444C45525F4D495353494EB0
:10BEC000470000004E52465F4552524F525F534F5B
:10BED00046544445564943455F4E4F545F454E4195
:10BEE000424C4544000000004E52465F4552524FBE
:10BEF000525F494E5445524E414C00004E52465FEF
:10BF00004552524F525F4E4F5F4D454D000000006D
:10BF10004E52465F4552524F525F4E4F545F464F0E
:10BF2000554E44004E52465F4552524F525F4E4F5F
:10BF3000545F535550504F52544544004E52465F43
:10BF40004552524F525F494E56414C49445F504111
:10BF500052414D004E52465F4552524F525F494E3C
:10BF600056414C49445F5354415445004E52465F3C
:10BF70004552524F525F494E56414C49445F4C45E1
:10BF80004E475448000000004E52465F4552524F03
:10BF9000525F494E56414C49445F464C414753001D
:10BFA0004E52465F4552524F525F494E56414C49A0
:10BFB000445F4441544100004E52465F4552524F47
:10BFC000525F444154415F53495A45004E52465FC7
:10BFD0004552524F525F54494D454F555400000051
:10BFE0004E52465F4552524F525F4E554C4C0000E8
:10BFF0004E52465F4552524F525F464F524249445D
:10C0000044454E004E52465F4552524F525F494E94
:10C0100056414C49445F4144445200004E52465FF1
:10C020004552524F525F4255535900004E52465F9F
:10C030004552524F525F434F4E4E5F434F554E5401
:10C04000000000004E52465F4552524F525F52452B
:10C05000534F5552434553004E52465F4552524F3F
:10C06000525F4D4F44554C455F4E4F545F494E49CA
:10C070005449414C495A4544000000004E52465F25
:10C080004552524F525F4D555445585F494E4954A1
:10C090005F4641494C4544004E52465F4552524F1F
:10C0A000525F4D555445585F4C4F434B5F46414995
:10C0B0004C4544004E52465F4552524F525F4D55DB
:10C0C0005445585F554E4C4F434B5F4641494C4594
:10C0D000440000004E52465F4552524F525F4D554C
:10C0E0005445585F434F4E445F494E49545F464163
:10C0F000494C4544000000004E52465F4552524FA5
:10C10000525F4D4F44554C455F414C524541445957
:10C110005F494E495449414C495A4544000000008A
:10C120004E52465F4552524F525F53544F52414711
:10C13000455F46554C4C00004E52465F4552524FAB
:10C14000525F4150495F4E4F545F494D504C454DF1
:10C15000454E5445440000004E52465F4552524FF2
:10C16000525F464541545552455F4E4F545F454ED0
:10C1700041424C45440000004E52465F4552524FEA
:10C18000525F494F5F50454E44494E470000000002
:10C190004E52465F4552524F525F4452565F54577B
:10C1A000495F4552525F4F56455252554E0000006E
:10C1B0004E52465F4552524F525F4452565F54575B
:10C1C000495F4552525F414E41434B004E52465FDC
:10C1D0004552524F525F4452565F5457495F455241
:10C1E000525F444E41434B004E52465F4552524FC0
:10C1F000525F424C455F495053505F52585F504B1D
:10C20000545F5452554E4341544544004E52465F8C
:10C210004552524F525F424C455F495053505F4325
:10C2200048414E4E454C5F414C52454144595F4553
:10C2300058495354530000004E52465F4552524FE6
:10C24000525F424C455F495053505F4C494E4B5FE3
:10C25000444953434F4E4E4543544544000000006B
:10C260004E52465F4552524F525F424C455F4950D5
:10C2700053505F504545525F52454A4543544544EB
:10C28000000000000000000098BE02000100000055
:10C29000A4BE020002000000C4BE020003000000B1
:10C2A000E8BE020004000000FCBE02000500000021
:10C2B00010BF02000600000024BF020007000000BB
:10C2C0003CBF02000800000054BF0200090000004B
:10C2D0006CBF02000A00000088BF02000B000000D3
:10C2E000A0BF02000C000000B8BF02000D0000005B
:10C2F000CCBF02000E000000E0BF02000F000000F3
:10C30000F0BF02001000000004C002001100000095
:10C310001CC00200120000002CC00200130000002C
:10C3200044C002008000000058C0020081000000EC
:10C330007CC002008200000098C002008300000060
:10C34000B4C0020084000000D4C0020085000000D8
:10C35000F8C002008600000020C10200900000002A
:10C3600038C102009100000058C102009200000094
:10C3700078C102000082000090C10200018200002A
:10C38000B0C1020002820000CCC1020000840000A3
:10C39000E8C10200018400000CC202000284000017
:10C3A00038C202000384000060C20200556E6B6E4A
:10C3B0006F776E206572726F7220636F6465000024
:10C3C0000100000001000000010000000100000069
:10C3D0000000010111121314636C6F636B00000005
:10C3E000434C4F434B0000004750494F5445000019
:10C3F00050525300554152540000000055415254D0
:10C400004500000053656E6420627574746F6E2081
:10C410007374617465206368616E67652E00000047
:10C420005265636569766564204C4544204F4E2112
:10C43000000000005265636569766564204C4544E0
:10C44000204F464621000000436F6E6E65637465A1
:10C4500064000000446973636F6E6E6563746564A5
:10C46000000000004E6F726469635F426C696E6B1E
:10C4700079000000426C696E6B79206578616D709F
:10C480006C6520737461727465642E0073645F62FE
:10C490006C655F6761705F646174615F6C656E6736
:10C4A00074685F75706461746528292028726571ED
:10C4B0007565737429206F6E20636F6E6E6563748B
:10C4C000696F6E20307825782072657475726E659C
:10C4D000642025732E000000546865207265717514
:10C4E00065737465642054582F5258207061636BD3
:10C4F0006574206C656E67746820697320746F6F53
:10C50000206C6F6E672062792025752F2575206F4E
:10C5100063746574732E00005468652072657175CC
:10C52000657374656420636F6D62696E6174696FB1
:10C530006E206F6620545820616E6420525820701F
:10C5400061636B6574206C656E67746873206973D2
:10C5500020746F6F206C6F6E6720627920257520C4
:10C560006D6963726F7365636F6E64732E00000094
:10C5700073645F626C655F67617474635F65786341
:10C5800068616E67655F6D74755F726571756573FF
:10C590007428292072657475726E65642025732E67
:10C5A0000000000073645F626C655F6761747473A0
:10C5B0005F65786368616E67655F6D74755F7265EE
:10C5C000706C7928292072657475726E65642025F7
:10C5D000732E00006E72665F626C655F67617474D3
:10C5E0000000000023D1BCEA5F782315DEEF1212B1
:10C5F0000000000001000007D0C90200D0C90200FD
:10C6000008000000D0C90200D8C9020008000000DC
:10C610006E72665F73646800D8C90200E8C90200E0
:10C6200008000000A0C90200D0C9020008000000F4
:10C6300073645F626C655F6366675F736574282906
:10C640002072657475726E65642025732077686545
:10C650006E20617474656D7074696E6720746F20EC
:10C6600073657420424C455F434F4E4E5F434647CF
:10C670005F4741502E00000073645F626C655F632A
:10C6800066675F73657428292072657475726E65BC
:10C6900064202573207768656E20617474656D7001
:10C6A00074696E6720746F2073657420424C455F17
:10C6B0004741505F4346475F524F4C455F434F559C
:10C6C0004E542E0073645F626C655F6366675F73D0
:10C6D000657428292072657475726E6564202573EF
:10C6E000207768656E20617474656D7074696E671B
:10C6F00020746F2073657420424C455F434F4D4D4D
:10C700004F4E5F4346475F56535F555549442E0091
:10C7100073645F626C655F6366675F736574282925
:10C720002072657475726E65642025732077686564
:10C730006E20617474656D7074696E6720746F200B
:10C7400073657420424C455F47415454535F4346E0
:10C75000475F415454525F5441425F53495A452EFA
:10C760000000000073645F626C655F6366675F73FF
:10C77000657428292072657475726E65642025734E
:10C78000207768656E20617474656D7074696E677A
:10C7900020746F2073657420424C455F47415454A8
:10C7A000535F4346475F534552564943455F4348AD
:10C7B000414E4745442E0000496E737566666963B5
:10C7C00069656E742052414D20616C6C6F636174B9
:10C7D000656420666F722074686520536F667444C8
:10C7E00065766963652E00004368616E6765207435
:10C7F00068652052414D207374617274206C6F63C0
:10C800006174696F6E2066726F6D203078257820B4
:10C81000746F20307825782E000000004D61786913
:10C820006D756D2052414D2073697A6520666F7277
:10C83000206170706C69636174696F6E2069732028
:10C84000307825782E00000073645F626C655F6548
:10C850006E61626C6528292072657475726E6564FC
:10C860002025732E000000006E72665F7364685F9F
:10C87000626C650098C90200A0C9020008000000AF
:10C880006E72665F7364685F736F630000202020C0
:10C890002020202020202828282828202020202070
:10C8A0002020202020202020202020202088101040
:10C8B000101010101010101010101010100404049C
:10C8C000040404040404041010101010101041415A
:10C8D0004141414101010101010101010101010148
:10C8E000010101010101010110101010101042425C
:10C8F0004242424202020202020202020202020218
:10C9000002020202020202021010101020000000B7
:10C910000000000000000000000000000000000017
:10C920000000000000000000000000000000000007
:10C9300000000000000000000000000000000000F7
:10C9400000000000000000000000000000000000E7
:10C9500000000000000000000000000000000000D7
:10C9600000000000000000000000000000000000C7
:10C9700000000000000000000000000000000000B7
:10C980000000000000000000000000000043000064
:08C99000382300200000000024
:08C99800D18C02000000000038
:10C9A0002DAD020000000000D1B202008C2B00204F
:10C9B000ADAA02000000000079B50200A02B002003
:10C9C00061B60200542B0020A1A10200000000006B
:08C9D000F98C020000000000D8
:10C9D800F9B802000000000065BB0200000000007A
:10C9E80070290020682900207029002028280020AC
:04C9F8001800000023
:10C9FC00E0C3020000000000E8C3020000000000D9
:10CA0C00F0C3020000000000F4C3020000000000AC
:10CA1C00FCC3020000000000CCBC020000000303B9
:10CA2C00C0BD020000000000F8BD020000000000C4
:10CA3C00D8C3020000000000D4C5020000000303AC
:10CA4C0010C602000000030368C8020000000303C4
:10CA5C0080C802000000030374BE02000000000046
:08CA6C008CBE02000000000076
:10CA740098BC020000000000A4BC020004230020B3
:08CA8400D897FF7F01000000BC
:10CA8C0000000000002000400000000000200040DA
:10CA9C000000000000000000FF000000001001403A
:10CAAC00110004000090D0030D00030001A102004E
:10CABC00FFFFFF00AC2B00201F0000006C2B0020A0
:10CACC001F0000008CC802000000000000000000E5
:10CADC00000000000000000000000000000000004A
:10CAEC0000000000000000008DC9020000000000E2
:10CAFC00000000000000000000000000000000002A
:10CB0C000000000000000000000000000000000019
:10CB1C000000000000000000000000000000000009
:10CB2C00000000000000000025620200016202000B
:04CB3C0000000000F5
:04000003200062D1A6
:00000001FF
